:020000040000fa
:080000000002040000000000f2
:020000040000fa
:04000800e20300000f
:020000040000fa
:04000c00fc030000f1
:020000040000fa
:04001000ae0300003b
:020000040000fa
:0400140016040000ce
:020000040000fa
:0400180030040000b0
:020000040000fa
:04001c007a03000063
:020000040000fa
:04002000c803000011
:020000040000fa
:040024009403000041
:020000040000fa
:04002800d8040000f8
:020000040000fa
:04002c006a04000062
:020000040000fa
:04003000d8040000f0
:020000040000fa
:04003400d8040000ec
:020000040000fa
:04003800d8040000e8
:020000040000fa
:04003c00d8040000e4
:020000040000fa
:04004000d8040000e0
:020000040000fa
:04004400d8040000dc
:020000040000fa
:04004800d8040000d8
:020000040000fa
:04004c00d8040000d4
:020000040000fa
:04005000d8040000d0
:020000040000fa
:04005400d8040000cc
:020000040000fa
:04005800d8040000c8
:020000040000fa
:04005c00d8040000c4
:020000040000fa
:04006000d8040000c0
:020000040000fa
:04006400d8040000bc
:020000040000fa
:04006800d8040000b8
:020000040000fa
:04006c00d8040000b4
:020000040000fa
:04007000d8040000b0
:020000040000fa
:04007400d8040000ac
:020000040000fa
:04007800d8040000a8
:020000040000fa
:04007c00d8040000a4
:020000040000fa
:04008000d8040000a0
:020000040000fa
:04008400d80400009c
:020000040000fa
:04008800d804000098
:020000040000fa
:04008c00d804000094
:020000040000fa
:04009000d804000090
:020000040000fa
:04009400d80400008c
:020000040000fa
:04009800d804000088
:020000040000fa
:04009c00d804000084
:020000040000fa
:0400a000d804000080
:020000040000fa
:0400a400d80400007c
:020000040000fa
:0400a800d804000078
:020000040000fa
:0400ac00d804000074
:020000040000fa
:0400b000d804000070
:020000040000fa
:0400b400d80400006c
:020000040000fa
:0400b800d804000068
:020000040000fa
:0400bc00d804000064
:020000040000fa
:0400c000d804000060
:020000040000fa
:0400c400d80400005c
:020000040000fa
:0400c800d804000058
:020000040000fa
:0400cc00d804000054
:020000040000fa
:0400d000d804000050
:020000040000fa
:0400d400d80400004c
:020000040000fa
:0400d800d804000048
:020000040000fa
:0400dc00d804000044
:020000040000fa
:0400e000d804000040
:020000040000fa
:0400e400d80400003c
:020000040000fa
:0400e800d804000038
:020000040000fa
:0400ec00d804000034
:020000040000fa
:0400f000d804000030
:020000040000fa
:0400f400d80400002c
:020000040000fa
:0400f800d804000028
:020000040000fa
:0400fc00d804000024
:020000040000fa
:04010000d80400001f
:020000040000fa
:04010400d80400001b
:020000040000fa
:04010800d804000017
:020000040000fa
:04010c00d804000013
:020000040000fa
:04011000d80400000f
:020000040000fa
:04011400d80400000b
:020000040000fa
:04011800d804000007
:020000040000fa
:04011c00d804000003
:020000040000fa
:04012000d8040000ff
:020000040000fa
:04012400d8040000fb
:020000040000fa
:04012800d8040000f7
:020000040000fa
:04012c00d8040000f3
:020000040000fa
:04013000d8040000ef
:020000040000fa
:04013400d8040000eb
:020000040000fa
:04013800d8040000e7
:020000040000fa
:04013c00d8040000e3
:020000040000fa
:04014000d8040000df
:020000040000fa
:04014400d8040000db
:020000040000fa
:04014800d8040000d7
:020000040000fa
:04014c00d8040000d3
:020000040000fa
:04015000d8040000cf
:020000040000fa
:04015400d8040000cb
:020000040000fa
:04015800d8040000c7
:020000040000fa
:04015c00d8040000c3
:020000040000fa
:04016000d8040000bf
:020000040000fa
:04016400d8040000bb
:020000040000fa
:04016800d8040000b7
:020000040000fa
:04016c00d8040000b3
:020000040000fa
:04017000d8040000af
:020000040000fa
:04017400d8040000ab
:020000040000fa
:04017800d8040000a7
:020000040000fa
:04017c00d8040000a3
:020000040000fa
:04018000d80400009f
:020000040000fa
:04018400d80400009b
:020000040000fa
:04018800d804000097
:020000040000fa
:04018c00d804000093
:020000040000fa
:04019000d80400008f
:020000040000fa
:04019400d80400008b
:020000040000fa
:040198004a04000015
:020000040000fa
:04019c00d804000083
:020000040000fa
:0401a000d80400007f
:020000040000fa
:0401a400d80400007b
:020000040000fa
:0401a800d804000077
:020000040000fa
:0401ac00d804000073
:020000040000fa
:0401b000d80400006f
:020000040000fa
:0401b400d80400006b
:020000040000fa
:0401b800d804000067
:020000040000fa
:0401bc00d804000063
:020000040000fa
:0401c000d80400005f
:020000040000fa
:0401c400d80400005b
:020000040000fa
:0401c800d804000057
:020000040000fa
:0401cc00d804000053
:020000040000fa
:0401d000d80400004f
:020000040000fa
:0401d400d80400004b
:020000040000fa
:0401d800d804000047
:020000040000fa
:0401dc00d804000043
:020000040000fa
:0401e000d80400003f
:020000040000fa
:0401e400d80400003b
:020000040000fa
:0401e800d804000037
:020000040000fa
:0401ec00d804000033
:020000040000fa
:0401f000d80400002f
:020000040000fa
:0401f400d80400002b
:020000040000fa
:0401f800d804000027
:020000040000fa
:0401fc00d804000023
:020000040000fa
:04020000d80400001e
:020000040000fa
:04020400d80400001a
:020000040000fa
:04020800d804000016
:020000040000fa
:04020c00d804000012
:020000040000fa
:04021000d80400000e
:020000040000fa
:04021400d80400000a
:020000040000fa
:04021800d804000006
:020000040000fa
:04021c00d804000002
:020000040000fa
:04022000d8040000fe
:020000040000fa
:04022400d8040000fa
:020000040000fa
:04022800d8040000f6
:020000040000fa
:04022c00d8040000f2
:020000040000fa
:04023000d8040000ee
:020000040000fa
:04023400d8040000ea
:020000040000fa
:04023800d8040000e6
:020000040000fa
:04023c00d8040000e2
:020000040000fa
:04024000d8040000de
:020000040000fa
:04024400d8040000da
:020000040000fa
:04024800d8040000d6
:020000040000fa
:04024c00d8040000d2
:020000040000fa
:04025000d8040000ce
:020000040000fa
:04025400d8040000ca
:020000040000fa
:04025800d8040000c6
:020000040000fa
:04025c00d8040000c2
:020000040000fa
:04026000d8040000be
:020000040000fa
:04026400d8040000ba
:020000040000fa
:04026800d8040000b6
:020000040000fa
:04026c00d8040000b2
:020000040000fa
:04027000d8040000ae
:020000040000fa
:04027400d8040000aa
:020000040000fa
:04027800d8040000a6
:020000040000fa
:04027c00d8040000a2
:020000040000fa
:04028000d80400009e
:020000040000fa
:04028400d80400009a
:020000040000fa
:04028800d804000096
:020000040000fa
:04028c00d804000092
:020000040000fa
:04029000d80400008e
:020000040000fa
:04029400d80400008a
:020000040000fa
:04029800d804000086
:020000040000fa
:04029c00d804000082
:020000040000fa
:0402a000d80400007e
:020000040000fa
:0402a400d80400007a
:020000040000fa
:0402a800d804000076
:020000040000fa
:0402ac00d804000072
:020000040000fa
:0402b000d80400006e
:020000040000fa
:0402b400d80400006a
:020000040000fa
:0402b800d804000066
:020000040000fa
:0402bc00d804000062
:020000040000fa
:0402c000d80400005e
:020000040000fa
:0402c400d80400005a
:020000040000fa
:0402c800d804000056
:020000040000fa
:0402cc00d804000052
:020000040000fa
:0402d000d80400004e
:020000040000fa
:0402d400d80400004a
:020000040000fa
:0402d800d804000046
:020000040000fa
:0402dc00d804000042
:020000040000fa
:0402e000d80400003e
:020000040000fa
:0402e400d80400003a
:020000040000fa
:0402e800d804000036
:020000040000fa
:0402ec00d804000032
:020000040000fa
:0402f000d80400002e
:020000040000fa
:0402f400d80400002a
:020000040000fa
:0402f800d804000026
:020000040000fa
:0402fc00d804000022
:020000040000fa
:04030000d80400001d
:020000040000fa
:04030400d804000019
:020000040000fa
:04030800d804000015
:020000040000fa
:04030c00d804000011
:020000040000fa
:04031000d80400000d
:020000040000fa
:04031400d804000009
:020000040000fa
:04031800d804000005
:020000040000fa
:04031c00d804000001
:020000040000fa
:04032000d8040000fd
:020000040000fa
:04032400d8040000f9
:020000040000fa
:04032800d8040000f5
:020000040000fa
:04032c00d8040000f1
:020000040000fa
:100400002f7121000eff24000e0188000000000063
:10041000000020000000e000020032000001200087
:100420002002880014000700630107000000e000bc
:1004300003003a0020f421000100200002003700f0
:100440000000200001002000810f70000100320038
:100450000f000700000020000000e0000200320052
:1004600000000200000000008c50020000000000ac
:100470000040da000000fe00000120000000e00063
:1004800002003200002020009001880000000600d9
:10049000a1028800800478000000eb001f003700f4
:1004a000e284440054a0b4009905ba00e2844400f8
:1004b00054a0b4009906ba00e284440054a0b400e9
:1004c0000006eb00476fde00fd07b200ae018800ba
:1004d000636ce10003003a000ad801000000eb0061
:1004e0000e003700606ce10008003a00004deb00a0
:1004f0000a05e800020039003420ec000af0a000f0
:100500008b05e900f9ff3e00040037006168e10057
:10051000010032000086eb000b00070019c7ba008b
:100520001905ba000e04e00003003a000a00e000da
:10053000dbff3a0000000600fe07b200ae028800b2
:100540008a047800f5ff37000cd0a300e20f4d00bd
:100550001c00390089027800354dba000a05e80010
:10056000020039003420ec000af0a0008b05e900fd
:100570000f003200254dba000a05e80002003900dc
:100580003420ec000af0a0008b05e90008003200de
:100590000c00e0000600320015cdba000a05e800a4
:1005a000020039003420ec000af0a0008b05e900bd
:1005b0008984e80054a0b4000b00e000e2ff3a0098
:1005c000000006009902ba00055d78008b05e9007d
:1005d000f7ff3200c82ade00055d78008b05e900d0
:1005e000f3ff32000c00e000f1ff320019ddba0029
:1005f000eeff370034510400000000001e510400db
:1006000000000000622e04000000000026390400f3
:10061000000000009439040000000000ac39040020
:10062000000000000e3a040000000000a02f0400ab
:1006300000000000b63a040000000000ce3a0400ba
:10064000000000001e4f04000000000022480400cb
:1006500000000000e04d040000000000f846040027
:10066000000000009045040000000000304b040032
:1006700000000000484f040000000000de210400dc
:1006800000000000fc410400000000003a360400b5
:1006900000000000224d0400000000000c46040091
:1006a00000000000a24d040000000000ec31040036
:1006b000000000008c51040000000000f250040013
:1006c00000000000ee3a04000000000008510400a1
:1006d00000000000dc500400000000001250040084
:1006e000000000009c4f040000000000d8510400ee
:1006f000000000003600f800809fbe00829fbe0010
:10070000849fbe00869fbe00000820009026070040
:100710004f03be004f02be004f01be004f00be009f
:100720003600f900004006003600f800809fbe0049
:10073000829fbe00849fbe00869fbe0000082000ee
:10074000832607004f03be004f02be004f01be00cc
:100750004f00be003600f900004006003600f800e9
:10076000809fbe00829fbe00849fbe00869fbe0009
:1007700000042000762607004f03be004f02be0093
:100780004f01be004f00be003600f90000400600d9
:100790003600f800809fbe00829fbe00849fbe008e
:1007a000869fbe0000022000692607004f03be009e
:1007b0004f02be004f01be004f00be003600f900e0
:1007c000004006003600f800809fbe00829fbe00f9
:1007d000849fbe00869fbe00100020005c2607009c
:1007e0004f03be004f02be004f01be004f00be00cf
:1007f0003600f900004006003600f800809fbe0079
:10080000829fbe00849fbe00869fbe002000200005
:100810004f2607004f03be004f02be004f01be002f
:100820004f00be003600f900004006003600f80018
:10083000809fbe00829fbe00849fbe00869fbe0038
:1008400040002000422607004f03be004f02be00ba
:100850004f01be004f00be003600f9000040060008
:100860003600f800809fbe00829fbe00849fbe00bd
:10087000869fbe0080002000352607004f03be0083
:100880004f02be004f01be004f00be003600f9000f
:10089000004006003600f8003200f8003400f8008e
:1008a00010002000a00188000020200000d0fe00e1
:1008b0000030a800018f8000d08e80000100010070
:1008c0000b88a9003400f9003200f9003600f90065
:1008d000004006003600f8000800fa001000200072
:1008e000c0bf9f004e35a80082aa800093aa800056
:1008f00061014100e081490082aa880093aa880032
:100900000028a900d0bf9f000000eb00e0bf9f00bf
:10091000f0bf9f0082aa800093aa8000f2bf9f00d0
:10092000e0bf9f006fb89700da14e30012003600b2
:10093000644d21006fb897000000400000004200a5
:100940001000780020019000b0019000ffb89700df
:1009500002814000e08149002200980033009800a5
:100960006fb897000000e800e0bf9f006fb89700e5
:10097000da14e300efff3e005035ef005235ef0090
:100980000028a9005fb8970021002000010078002e
:10099000f1100700cfb9970003006000c0bf9f00af
:1009a0000c77ef000080fa003600f90000400600e6
:1009b0000040da000000fe00000005000001eb002e
:1009c00015000700040032000200200003f8230095
:1009d00001f0a6003b01070000000600839f6800ad
:1009e0000100e00002003d0060001000e0801800ff
:1009f0000300e00002003d0060011100e0811900e9
:100a0000580207004f00e00002003b0060001000a9
:100a1000e080180000000600889fbe008a9fbe008c
:100a20000003be0066000700850578008281520041
:100a3000020020006220e10004003a00f307b10048
:100a4000040035007718e100040035000600be0000
:100a5000140037006000b8000f003700f50f2000c9
:100a6000faff2f008502d1000a85d3008301e90037
:100a7000fcff3b008184620000046500890f740064
:100a8000f2ff32008582ea000a85ea008184620072
:100a9000000465002400070007f0a70001f0a00093
:100aa0000081eb000200e0004f05be004f04be00d5
:100ab000000006000001be00410007000470a7000e
:100ac00003f0a10003f8a30013003a006509b10088
:100ad00010003200090035006928e10002003500ed
:100ae000010028000000050000004000818048004f
:100af0008502e900fcff3a0000000600f88f420082
:100b0000050035008100d1000080d3008502e80097
:100b1000fcff3a00000006008000eb00000005002a
:100b20006011b800d00437008100200061805500ba
:100b30000b003d000b00200061fe2f000100e100d2
:100b40001d00340082817100610164008904d100bc
:100b50000884d3000000e800faff3a00710020008a
:100b600061006400030070000200600009003200b0
:100b700061044400e0844c000988a50005003200af
:100b80008b05e8006808e10002003a008904d10002
:100b90000884d300f20f20000258e10005003d0058
:100ba000c75ddd00f907b200898075000800780094
:100bb000000006000bf827008b00780000000500fd
:100bc000c70ade00f107b200f50fb20008003200dc
:100bd000e1cf4200020032000170a00024000500b5
:100be000810f700001003200040805004400050078
:100bf000810f700002003a00140005008502e90030
:100c00000000400081c04800fcff3b000170a000d4
:100c100024000500f2ff2f00010037000001eb0067
:100c2000850007000718a3006e0032000728a30004
:100c300002003a000738a3006a003200889fbe0015
:100c40008a9fbe008c9fbe008e1f78003200f80085
:100c5000082020009801880002077800820307001e
:100c6000020478000620200086844000ca4cde0082
:100c7000f08454006848e100010035000804e800f1
:100c80000001eb000900e0002100320026f92800f5
:100c900066c27c000482fb004622dd0004e0a00066
:100ca0000123b8000020b8008680400060814b001e
:100cb000060022000601510017020700010078001b
:100cc0008200780061811100060028000608e1001a
:100cd00004003a000000e00002003a0001002c008d
:100ce0000201e8000100e00001003a000001eb0011
:100cf0000006be0082057800670341000600e000a0
:100d000008003d0043002000e400290007003700f0
:100d1000050024000400200003002000b2030700a7
:100d2000f3ff370053002000a40029004a01070008
:100d30000c02be008b017800200307006f83640063
:100d4000060032004afa2800664bb8000605450046
:100d50003a02be009a017800a30307000800e000f1
:100d6000130032000006be0082057800c4bf2000d8
:100d7000958b25000440b8000543b80086804000ec
:100d800060814b0008f8a30002003200848050000c
:100d900005015900e0010700010078008200780099
:100da0006f8111000c02be008b01780090030700d8
:100db0000e00e0000400320054c52e00d5f22600db
:100dc000e3ff2f00fd020700d40307003200f90003
:100dd0004f0778004f06be004f05be004f04be000f
:100de000000006000778a30005003a000768a3008a
:100df000050032000718a3000300320000000600bf
:100e00000160a000090037000748a3000500320078
:100e10000718a300030032000000200001f82f0093
:100e200000000600f0ff2f00f1ff27001202200053
:100e300082b88800000006002700200001f0a7000b
:100e400017002000470bde00f60fb200040032004e
:100e50000643e8000a0032004702b3000000060023
:100e600001037800f607b2000603700002003a00a2
:100e70000703b300000006008702b300000006006d
:100e800001037800f607b20006037000020032008a
:100e90000770a000000006000760a0000000060028
:100ea00007f82700078361000638e10004003a00d4
:100eb000f7072000878361008703710001003a0073
:100ec00003f0a200889fbe008a9fbe008c9fbe00d8
:100ed000470ade000480a100c71ade000580a100d9
:100ee000070028000785600087856100f70f200054
:100ef0000720e1009e0032000728e1009c0032003c
:100f0000010678000400e000b4003200f70720007a
:100f1000878060000170a0000500e000c000320082
:100f2000f7072000878161000370a00005065200ca
:100f30000f003a000b50e1000b0032000308e10003
:100f400002003a000200e1007e003200020450007c
:100f500083845800040031000001fd008101fd0080
:100f60008402fd008a05fd006044b80021003700be
:100f70000520e10005003d000001fd008101fd00ac
:100f80008402fd008a05fd00050652007a60e1003a
:100f9000050035000170a1004722dd00848070004b
:100fa0008a807000630037006044b800ef0266007a
:100fb00007ff2f00070666000500e000060034006a
:100fc000f08312008714dd000511de00071bdd0031
:100fd000060171008519de007060e1000500350032
:100fe0000904780082047800030178008001eb0096
:100ff000700656000b50e10003003a00020040006a
:10100000838048000400370060041400e0841c0062
:1010100002005800838058000188a30006003200b7
:101020008100d1000080d3008984d3000884d300dc
:101030000402e800270037000178a30025003a00e9
:101040000100e000030032008186cf00698656006f
:101050000a0037008c0020000000e00004003a0085
:1010600009007800880478000004eb007002520048
:101070008086cf000d0646000c06e9007060e10096
:1010800006003500800078000900780088047800a8
:101090000004eb0070065600700252000c00e000e5
:1010a0000c0034008c08dd00f00316000703de009e
:1010b000868070000c00dd00074bde00060070002b
:1010c0008c4cdd000743de00868474000c44dd0098
:1010d0000c0252006120e100200035006101600037
:1010e0000700280087816400f7ff270087836400da
:1010f000070374000300e00006003200820373005f
:10110000040032000000e800e08048000188a300ed
:101110000e003a00f70f20000720e1004a003d00d2
:101120000170a1004722dd00810072008a807000fa
:101130000000be004f06be004f05be004f04be00bb
:10114000000006006000b800faff37008100d100ff
:101150000080d3000402e800eeff370004017800ad
:1011600089017400730207008a807000f1ff370064
:1011700031ff0700070278000001fd008101fd003a
:101180002dff070087027800850372000778a3000f
:10119000040032000001fd008101fd00fe01070096
:1011a000e4ff3700850362000768a30008003200ef
:1011b0000b50e10003003200f0ff2f00f1ff270089
:1011c000dcff37000001fd008101fd00d9ff370081
:1011d0000468a300d7ff3200faff3700f8ff2700aa
:1011e000888360000b003a000000e00009003a002c
:1011f0008303640082837300020032000200be0099
:10120000ccff37000b50e100ceff3a000200be00d9
:10121000c8ff370014002000810064003eff370043
:10122000f8ff27008883610004003a000200e00014
:1012300002003a008c007800beff37001500200045
:101240008301640039ff370001f827000000200007
:1012500081007500b7ff37006218e1003b003500e0
:10126000889fbe008a9fbe008c9fbe008301e9005c
:101270000004be000205be000406780062054500b9
:101280000a05ea003c00be007050e100170035007e
:101290000d0032007f50e10001003400fa0120000f
:1012a000f00655000801be00bf0007000d99de00e2
:1012b000cf99de003c004100bc8049008b05e9006d
:1012c000f8ff3c00140037000801be00b60007001c
:1012d00003017800cf99de003c004100bc8049004a
:1012e0008b05e900f8ff3c000b003700f006150005
:1012f0000801be00ac0007000a11de008d1add00f7
:10130000050171008a99de003c004100bc80490063
:101310008b05e900f6ff3c000103df000605ea004b
:10132000050034008a08dd00700215008402de002a
:10133000858070000a00dd00060178004f06be00bf
:101340004f05be004f04be00000006000300e00091
:1013500002003a006000b800020005003400be0040
:10136000020005000202500083825800610039002b
:10137000030371006200320005037200590032005d
:101380000300e0005500330017003a000100e000c0
:101390004b0032000208e1000600310005000900a0
:1013a0004288d800010178008001eb008000eb004a
:1013b000000006006110e100550032000002be008e
:1013c000050009008280d8008002780004007800bf
:1013d000050009004288d800010178008001eb0077
:1013e0008500780000000600889fbe008a9fbe002e
:1013f0008c9fbe000386cf000c06e9008c1f78008e
:101400008c19dd00f00216000512de0084817100e7
:101410000c11dd000003be008004eb00053cde0083
:101420008c3bdd000532de00848373000c33dd006d
:101430000700780088007800050009004388d8007c
:101440000202b8000306b8008c82420060854e009c
:101450008005eb000402530085825b000a055c00f6
:101460008b855c000b0033008000eb004f0678009a
:101470000c21de00700516000a2ddd000a01710046
:101480008c29de004f06be004f05be004f04be0093
:10149000000006000202420083824a0060054d00ff
:1014a000e0854d000000e9000b00e000eeff3d008c
:1014b0000202420083824a000000e900eaff37008e
:1014c0000000e00012003200050009000280d80090
:1014d000010178008000eb00000006000401be005e
:1014e000010037006011b800100020008000eb0000
:1014f000000006000001be006000b8000000060009
:101500000001be00f0ff2f00f1ff2f0000000600d9
:101510006011b800000006008001eb000202df004d
:101520000402ea006f20e10010003a000201d1003d
:101530000181d3008080d3004f00dd00f300200044
:101540000202df000402ea006f20e10007003a0017
:101550000201d1000181d3008080d3000000eb00a4
:10156000e30120000202df000402ea000400e000c0
:1015700009003200f00212000411dd00050bde004c
:10158000060171008408dd000503de00868070001e
:101590000400dd00848141000200e000010032000f
:1015a0000000060003000500889fbe008a9fbe0061
:1015b0008c1f78000002be000203be000620b800a7
:1015c000062db8008a80400060814d000724b800d5
:1015d000072db8008a84440060864d0081004400d5
:1015e00002814c00e0014e000700e00008003500d9
:1015f0000500e00002003d0006015100878159000e
:101600004f0678004f05be004f04be0000000600e4
:101610000401510085815900f5ff3700889fbe0005
:101620008a9fbe008c9fbe001b0020000202be00ed
:101630000586680006002800060666004709de00e9
:10164000f20fb200820032000243e8008000320054
:10165000c729de00f30fb2007d0032000343e8002b
:101660007b003200f107b2000170a000f507b20064
:101670000570a000c708dd004903de008680700009
:101680004700dd00c72add004923de0086827200a4
:101690004722dd00030551000403500085835800f4
:1016a0000300310000004000818048000a05e90085
:1016b0008c1f78008a9fbe0004005000858058006f
:1016c0000402420085824a000000400081804800f8
:1016d0000005eb000004be006033b8000406be0045
:1016e0000d48e10056003100050009004dccd8003e
:1016f0000c01b8000d02b8008481410060824a00ec
:101700008283530003045c0084845c0060055d00f8
:101710000a00e00025003a00800578000d40e10055
:1017200049003100880078000700780005000900b2
:101730004d88d8000c01b8000d02b800848141002a
:1017400060824a006003110083835b0004045c0034
:10175000e0845c000900e00021003a004f01be0077
:101760000300e0002b003200e30160000706730075
:101770008c81710001003200640070004200de00c4
:101780004e5edd000c007000c258de0001e0a000db
:1017900062010700cf017800818071004f06be0012
:1017a0004f05be004f04be00000006008c834300be
:1017b0000d044c00e0844c0060054d000000e90081
:1017c0000a00e000d4ff32008c8343000d044c007b
:1017d000e0844c0060054d000000e900ceff3700ba
:1017e0000c0343008d834b0060044c00e0844c00ec
:1017f0000000e9000900e000d8ff32000c034300bc
:101800008d834b0060044c00e0844c000000e90034
:10181000d2ff37004200de004e5edd000c0070009b
:10182000c258de0001e0a000cf0178000300e00014
:10183000daff320060001000e0801800d7ff3700a8
:10184000f0ff2f00aaff3700f0ff2f00b9ff37008d
:101850000404be0078fd0700870678000004fd0040
:101860008104fd0074fd0700078366000678a3006d
:10187000030032000960a7000800be002c003700fa
:101880000d78a300020032000800be0028003700d7
:101890000778a30026003a0001f0a10009f0a1009a
:1018a0000668a30003003200f1ff2700f0ff2f00bd
:1018b000baff37000d68a300030032000800be0025
:1018c0008c807000b5ff37000768a30007003a005e
:1018d0000648a30003003200f1ff2700f0ff2f00ad
:1018e000aeff37000d48a300030032006000b800cf
:1018f0008c807000a9ff37000748a3000400320065
:1019000001f82700000020008c807000a3ff370042
:10191000550007000004fd008104fd000205780069
:10192000510007000802be008a01780059ff370005
:101930000160a0001202200082b8880097ff3700e3
:101940000100e000120032000500e000100032004b
:10195000889fbe008a9fbe008c9fbe000006eb00e1
:1019600001f8a3000300320060001000e0801800be
:101970000cf0a00005f8a300030032006002120082
:10198000e0821a000cf0a2008005eb0041ff370056
:101990006000b800020005000478a30004003200d3
:1019a0000578a300030032000168a30001003a009b
:1019b0000200be000160a00000000600889fbe007b
:1019c0008a9fbe000004be000405be000301410062
:1019d0000201e8008000eb000a42b8000b43b800a7
:1019e0008682420060804b000a4bb800868242002b
:1019f00007004800e08048000b4bb800060040009c
:101a0000878048000103700002003a000001eb00eb
:101a1000120037000900e00002003d000a005000fb
:101a20008b8058000b00e00002003d0008005000d1
:101a3000898058008582420000004800818048006b
:101a40008101df000300e0000400320085824200d3
:101a500000004800818048000201e9004f05be00f7
:101a60004f04be00000006004f0ade004709de00fa
:101a7000f107b200f20fb2000b003200f207b10022
:101a80000170a000c708dd00c901de00838070007e
:101a90004700dd000400a600000006006000100002
:101aa000e080180000000600810f700001003a007d
:101ab000000006008182cf000500e00010003e001b
:101ac0008082cf00ee8242007028e10004003900dd
:101ad00007003e00800078000000eb000e00370099
:101ae000708312008600de000500dd000a0037006a
:101af000708352008600dd000000eb000600370016
:101b0000e28252008508dd00708312000603de00c9
:101b1000868070000500dd007507b0000501ea0051
:101b20000400a6000000060060001000e08018001d
:101b3000000006000100e0002600320061011100f3
:101b40007810e10023003c006022b8007010e10032
:101b50000400350080027800010078008000eb006e
:101b6000700151000200e000090034007003110010
:101b7000062add00822ade008603dd0087827200ed
:101b80000200de00860bdd00070070008208de0028
:101b900084817100f4ff2700048262008481710057
:101ba00004002800848262006102600005f0a60043
:101bb0000000060004827100070032000000e80007
:101bc000e0804800000006000002be006000b8008f
:101bd000efff37006000b800000006006000100052
:101be000e08018000200370060021200e0821a0054
:101bf0000100e0003f0032000500e0003900320043
:101c0000889fbe008a9fbe00820378008304510033
:101c100004003d000002fd008102fd008904ea008d
:101c20008303780001017800800078000000eb0059
:101c300005037800840278000002eb0006056900c5
:101c4000070035000281d1008180d3000080d300dd
:101c50000683d1008582d3000482d3008703e80085
:101c60007048e100060035007f48e10029003c0093
:101c700005027800860278004fb3de00f08454003d
:101c80000900e000080032000922de00708514001f
:101c90008a2ddd000b027200892ade008a35dd0004
:101ca0008b82720009b3de0004004000858048008a
:101cb0000601490018fe0700838353000200e0007c
:101cc000090032000b0028000b10e1000c0032006c
:101cd0000100780082007800070178004f05be00ff
:101ce0004f04be00000006006000b8000001eb00d9
:101cf000faff37000400be00030178000000060070
:101d00000100e000f2ff3a0002002c008703e80027
:101d1000efff3700f9012000d5ff37008101700087
:101d2000270032008002eb0001f8a300030032001c
:101d300060001000e080180015002000f40720006b
:101d40000202420020003400f703200087036000f5
:101d50000604200000036300020820000001610067
:101d60004700de00c909dd0000807100c708de0001
:101d70000600e00008003200870371000600320010
:101d80001000b0000180b0000188a3000200320002
:101d9000c108de000402e800f107b200f30f2000e2
:101da0000320e10003003d004722dd0081007200b6
:101db0002900370001f827000000eb00260037005b
:101dc0006000b80000000600680212007f20e100f9
:101dd000020034006000b8001f0037006011b80036
:101de0007020e100040035008001780001007800d7
:101df0008000eb00700252000400e0000900340093
:101e0000f00312000719dd008419de000703dd006e
:101e1000868171000400de00070bdd000600700003
:101e20008408de00f7ff27008383630087037100c7
:101e30000600280003036300070032000700e000eb
:101e400003003a0061016000028173000200320069
:101e50001000b0000180b0000500a60000000600e0
:101e600001f0a00000000600889fbe008a9fbe000f
:101e700000827000040271000482710026003200aa
:101e80000004be000200be006011b8006b09200013
:101e9000950220000182cf000a0039000541b100ff
:101ea0000082cf00070039000541b1000982cf0050
:101eb000040039000541b1000882cf00010039005b
:101ec0000541b10005425200120032000a003b00f9
:101ed00082817100610164008100d1000080d30023
:101ee0008984d3000884d3008b05e8000442e8000d
:101ef000f7ff3a00070037000804440089844c00cb
:101f000000004800818048008b05e9000442e90098
:101f1000f9ff3a0004fb07004f05be004f04be0066
:041f200000000600b7
:020000040000fa
:101f240000e20000c7af00009a860000746400005d
:101f3400554800003b2f0000251a0000110800003e
:101f4400000000000000000000000000000000008d
:101f54000039000057840000fbff000048e0000047
:101f640023870000fcff0000fe3b0000d3a7000015
:101f7400fdff0000e4100000408e0000fdff0000a3
:101f8400d28c000052ba0000feff0000f6c8000028
:101f940039ae0000feff0000249e0000f8a20000fd
:101fa400feff00004480000065490000feff0000c1
:101fb400b6610000e47e0000fdff0000f2b3000003
:101fc4002f6a0000fdff000066e300004c5600008d
:101fd400fdff0000121600001e450000fdff00007a
:101fe400581700000d630000fcff0000d6600000dd
:101ff400d6410000fcff00003a6c00000a7e00009d
:10200400faff0000000000000000000000000000d3
:10201400b9650000cf0c000046f80000fcef00009a
:102024002f550000551500002c00000000e00000b2
:08203400000000000040000064
:020000040000fa
:10203c00e2140000dc140000d6140000e8140000c8
:10204c00e6140000e0140000da140000ec140000a8
:020000040000fa
:10205c00e8874700889fbe008a9fbe008c9fbe0009
:10206c008e1f78001b002000ebb79f007c10f8003f
:10207c00d211f900c03b2000808e880080fc2f001c
:10208c00b08e8800f0412000c08e8800809820001f
:10209c00a08e8800202f2100d08e880021e62200ff
:1020ac00e18e880061922300018f88004199230002
:1020bc00f18e8800c19a2300118f8800e18e800078
:1020cc0001000100d08e800021c220002041900030
:1020dc000044eb0021409800c808de00304190001d
:1020ec0031409800d08e80008048900008489800bd
:1020fc009048900018489800d08e8000c040900006
:10210c0053c0b30043409800d04090005840980012
:10211c00d08e8000e0409000f2c9b300624098007d
:10212c00f0409000e1c4b30071409800d08e800064
:10213c0004c22000fc0f2000a04a90002448980004
:10214c004822de00b04a900034489800d08e8000bf
:10215c0000529000085098001052900018509800af
:10216c00d08e8000404a900043489800d04990009f
:10217c0058489800d08e8000e04990006248980042
:10218c007049900071489800d08e8000411e21004b
:10219c000c81600082bf9f00205190008ff197004e
:1021ac0023509800c808de00f1b79f00b050900093
:1021bc00efe8970031509800d08e80008058900046
:1021cc00085898009058900018589800d08e8000ad
:1021dc00c050900048509800d05090005850980033
:1021ec00d08e8000e050900080c4eb0069509800c5
:1021fc00f0509000fac7b3007a509800d08e80004f
:10220c00811f21002059900021589800c808de0039
:10221c003059900031589800d08e8000806090002a
:10222c00086098009060900018609800d08e800034
:10223c00c058900048589800d058900058589800b2
:10224c00d08e8000e058900069589800f0589000ab
:10225c007a589800d08e8000011d210020619000da
:10226c0021609800c808de00306190003160980051
:10227c00d08e8000b18e800000c9900001c89800fb
:10228c00c808de0010c9900011c89800d08e8000dc
:10229c00c18e800020c9900021c89800c808de00bb
:1022ac0030c9900031c89800d08e8000c0c8900012
:1022bc0048c89800d0c8900058c89800d08e8000ac
:1022cc00e0c8900068c89800f0c8900078c89800e2
:1022dc00d08e80004e3520008c06670080d0900098
:1022ec000dd098004877de0090d090001ed098005a
:1022fc00d08e8000a0d0900028d09800b0d0900054
:10230c0038d09800d08e8000c0d090004dd098006e
:10231c00d0d090005ed09800d08e8000e0d090009d
:10232c0001ceb30061d09800f0d090007bd0980023
:10233c00d08e8000c104210000d9900001d89800f3
:10234c00c808de0010d9900011d89800d08e8000fb
:10235c008104210020d9900021d89800c808de0003
:10236c0030d9900031d89800d08e8000e104210043
:10237c0040d9900041d89800c808de0050d9900090
:10238c0051d89800d08e80000105210060d99000b2
:10239c0061d89800c808de0070d9900071d89800f8
:1023ac00db8e8000b08b2e00e10e2c0018fa07009b
:1023bc008221270013f3230095fc07007cf907000a
:1023cc00b9f90700f2ff27008090de002bc09000c7
:1023dc00a1c59800c808de003bc09000b1c59800ac
:1023ec00db8e8000b08b2e00e10e2c0008fa07006b
:1023fc008221270013f3230085fc07006cf90700ea
:10240c00a9f907008000ea000bc0900081c5980074
:10241c00c808de001bc0900091c59800db8e8000c0
:10242c00b08b2e00e10e2c00f9f907008221270059
:10243c0013f3230076fc07005df907009af90700f7
:10244c00a28120008090de004bc09000c1c5980096
:10245c00c808de005bc09000d1c59800d08e80000b
:10246c00e0c0900068c09800f0c0900078c0980060
:10247c00d08e800080e0900008e0980090e0900002
:10248c0018e09800d08e8000a0e0900028e0980022
:10249c00b0e0900038e09800d08e8000c0e0900052
:1024ac0048e09800d0e0900058e09800d08e800072
:1024bc00e0e0900068e09800f0e0900078e0980090
:1024cc00d08e800080e8900008e8980090e890009a
:1024dc0018e89800d08e8000a0e8900028e89800ba
:1024ec00b0e8900038e89800d08e8000c0e89000ea
:1024fc0048e89800d0e8900058e89800d08e80000a
:10250c00e0e8900068e89800f0e8900078e898001f
:10251c00d08e800080f0900008f0980090f0900031
:10252c0018f09800d08e8000a0f0900028f0980051
:10253c00b0f0900038f09800d08e8000e2a023001c
:10254c008c006100c0f1900041f09800c810de00d2
:10255c00d0f1900051f09800d18e8000e03721002e
:10256c000c066000e1f19000ecf09800c801de0070
:10257c0071f29000f3f09800d18e800081f99000f8
:10258c0088f8980091f9900098f89800d18e800006
:10259c00a1f99000a9f89800b1f99000baf8980048
:1025ac00d18e8000c1f99000c8f89800d1f9900044
:1025bc00d8f89800d18e8000e1f99000e8f89800e6
:1025cc00f1f99000f8f89800d18e800081419100cb
:1025dc00884099009141910098409900d18e8000db
:1025ec00a1419100a8409900b1419100b8409900d7
:1025fc00d18e8000c1419100c8409900d141910019
:10260c00d8409900d18e8000e1419100e8409900ba
:10261c00f1419100f8409900d18e800091419000d9
:10262c000374a10093409800d18e800091419000da
:10263c000354a10093409800d18e800091419000ea
:10264c000344a10093409800d18e800091419000ea
:10265c000364a10093409800d18e80001104a10066
:10266c00d18e80001114a100d18e80009141900078
:10267c000334a1009340980001782000318f88002a
:10268c00f3412000238f8800810c2000518f88009b
:10269c00012c2100618f880081dd2000418f880092
:1026ac00708f880001fa2200818f8800a28f880029
:1026bc0061ab2300918f8800e1ac2300b18f8800bf
:1026cc00818f800001000100708f8000e1c020002c
:1026dc002041900021409800c808de003041900055
:1026ec0031409800708f80008048900001c8b30082
:1026fc00014898001049900072c0b300124898002d
:10270c00708f8000c041900042409800d0419000f2
:10271c0058409800708f8000e0419000694098000c
:10272c00f041900033c6b30073409800708f800066
:10273c0084c22000a04a9000244898004822de0061
:10274c00b04a900034489800708f8000005290007e
:10275c00015098001052900012509800708f800019
:10276c00404a9000424898005049900058489800c0
:10277c00708f800060499000694898007049900003
:10278c0073489800708f8000e2342000a0519000b4
:10279c00225098004811de00b05190003250980041
:1027ac00708f8000005990000858980010599000c4
:1027bc0018589800708f8000405190004850980035
:1027cc005051900058509800708f800060519000cc
:1027dc0069509800705190007a509800708f80006a
:1027ec00a23b2000a0599000225898004811de000e
:1027fc00b059900032589800708f800000619000a2
:10280c00086098001061900018609800708f80002c
:10281c0040599000485898005059900058589800ca
:10282c00708f800060599000695898007059900022
:10283c007a589800708f8000206190000ff19700fb
:10284c002260980030619000efe9970033609800a7
:10285c00708f8000528f800080c9900002c8980051
:10286c004811de0090c9900012c89800708f80004b
:10287c00628f8000a0c9900022c898004811de0029
:10288c00b0c9900032c89800708f8000528f8000c1
:10289c00c0c9900042c898004811de00d0c9900011
:1028ac0052c89800708f8000628f8000e0c9900041
:1028bc0062c898004811de00f0c9900072c89800f8
:1028cc00708f800000d190000dd0980010d1900036
:1028dc001ed09800708f800020d1900082cdb30064
:1028ec0022d0980030d19000d2c0b30032d09800e2
:1028fc00708f8000023c2000c0d1900042d0980024
:10290c004811de00d0d1900052d09800708f80001a
:10291c0060d1900061d09800f0d09000c1c0b3009d
:10292c0071d09800708f800080d8900008d89800e3
:10293c0090d8900018d89800708f8000a0d8900084
:10294c0028d89800b0d8900038d89800708f8000a4
:10295c00c0d8900048d89800d0d8900058d898008b
:10296c00708f8000e0d8900068d89800f0d8900064
:10297c0078d89800708f800080e0900008e0980074
:10298c0090e0900018e09800708f8000a0e090001c
:10299c0028e09800b0e0900038e09800708f80003c
:1029ac00c0e0900048e09800d0e0900058e098001b
:1029bc00708f8000e0e0900068e09800f0e09000fc
:1029cc0078e09800708f800080e8900008e898000c
:1029dc0090e8900018e89800708f8000a0e89000b4
:1029ec0028e89800b0e8900038e89800708f8000d4
:1029fc00c0e8900048e89800d0e8900058e89800ab
:102a0c00708f8000e0e8900068e89800f0e8900093
:102a1c0078e89800708f800080f0900008f09800a3
:102a2c0090f0900018f09800708f8000a0f090004b
:102a3c0028f09800b0f0900038f09800708f80006b
:102a4c00c0f0900048f09800d0f0900058f098003a
:102a5c00718f800061f09000e8f0980071f09000a8
:102a6c0008407800f0f09800718f800021c1900030
:102a7c00a0c0980031c19000b0c09800718f800048
:102a8c0001c1900080c0980011c1900090c09800c6
:102a9c00718f800041c19000c0c0980051c190005e
:102aac00d0c09800718f800061c19000e0c0980088
:102abc0071c19000f0c09800718f800001f99000f6
:102acc0080f8980011f9900090f89800718f8000b0
:102adc0021f99000a0f8980031f99000b0f8980016
:102aec00708f8000c0f8900002c8b30042f89800c4
:102afc00d0f89000c1c0b30051f89800708f8000de
:102b0c00e0f9900062f8980070f9900071f8980064
:102b1c00708f8000613f20000041910001409900be
:102b2c00c808de001041910011409900708f8000a0
:102b3c00a13820002041910021409900c808de00f6
:102b4c003041910031409900708f8000013f20008e
:102b5c004041910041409900c808de00504191006d
:102b6c0051409900708f80004138200060419100e5
:102b7c0061409900c808de007041910071409900d5
:102b8c00708f8000904090000174a100114098005b
:102b9c00708f8000904090000154a100114098006b
:102bac00708f8000904090000144a100114098006b
:102bbc00708f8000904090000164a100114098003b
:102bcc00708f80001004a100708f80001014a10081
:102bdc00708f8000904090000134a100114098004b
:102bec00801f2100411e21000900090031187800c6
:102bfc0001782000d18f880000c82000e08f880069
:102c0c00c2202100431e210009000900331978005d
:102c1c00719088008090880002222100431e2100c0
:102c2c00090009003319780011918800209188005f
:102c3c006fb097004f0778004f06be004f05be00df
:0c2c4c004f04be008f00b1000000060025
:020000040000fa
:102c58000800fa00889fbe008a9fbe0080047800a2
:102c680010002000000f78000000eb00100798000b
:102c780010079800b91890001e009000808f50002f
:102c8800c40136004a0320001e0090008a80b90063
:102c98000080440060b09000200798001e0090005b
:102ca8008a80b9000080440070b090003007980016
:102cb8003e009000000040004123210000804000b9
:102cc80010007800e04090008180fb00f041900007
:102cd800c819dd00838170001e0190008a91b90037
:102ce8008280440001b99000110020000209dd0033
:102cf8000281ea0003016100e0419000624098000f
:102d08004811de00f0419000724098006042900047
:102d18000482fb00f0419000c819dd0083017200b5
:102d28001e0190008a91b9000281440012b99000f6
:102d38000209dd000281ea0003016100e041900020
:102d4800624098004811de00f041900072409800ff
:102d5800204290000482fb00b0419000c819dd00b9
:102d6800830172001e0190008a91b900028144001b
:102d780002b990000209dd000281ea000301610046
:102d8800a0419000224098004811de00b041900018
:102d980032409800204290000482fb00b04190002d
:102da800c819dd00830172001e0190008a91b900e4
:102db8000281440012b990000209dd000281ea0094
:102dc80003016100a0419000224098004811de00f4
:102dd800b041900032409800404a90000482fb00c5
:102de800d0499000c819dd00830172001e019000cf
:102df8008a91b9000281440002b990000209dd00fd
:102e080002817100c0499000424898004811de00d4
:102e1800d049900052489800c04990008381fb0037
:102e2800504990004811dd00028171001e02900097
:102e38008aa2b9008481440093b990008308dd0018
:102e4800810071004049900041489800c808de00a0
:102e580050499000514898002e0090000000e90069
:102e680000004000c1582100008040001004780094
:102e78001e0090008a80b9000080440060b0900075
:102e88006f03b000abfc2f008f85450081512100f6
:102e98001a000900b11d78006b03b1000f1c070070
:102ea8001e0f60001e0090008a80b9000080440058
:102eb800d0f09100e1c06000620020008208dd00cf
:102ec800384090000064a100014070003044980030
:102ed8001e0090008a80b9000080440060f09100d4
:102ee80061406000710020000100dd00984078001a
:102ef8000174a10000cc70001e0090008a80b90007
:102f08000080440070b89000c86090004064980049
:102f18004800de00d8609000506498001e009000c1
:102f28008a80b9000080440040b89000886890000a
:102f3800006c98004800de0098689000106c9800bb
:102f48001e0090008a80b900008044002000910093
:102f580088709000007498004800de009870900017
:102f6800107498001e0090008a80b9000080440008
:102f780010009100a8709000207498004800de00ae
:102f8800b8709000307498001e0090008a80b900d4
:102f98000080440030009100e8589000605c980080
:102fa8004800de00f8589000705c98001e00900001
:102fb8008b0778000000e00021003a0039189000e3
:102fc800e10f50001e003600384090000034a10088
:102fd80030449800a840900000cfb30000c06000c3
:102fe80020449800a848900080cfb30080c06000bb
:102ff8003140b300214c98001e0190000201e80006
:103008008a91b90082804400d1b890006869900024
:10301800616c9800c808de0078699000716c9800af
:10302800b840900000c060000004a0003044980040
:10303800284890008041b300204c98006f0037006a
:103048001e0090000000e0002a003200b91890002d
:103058001e0090008100e900808f50002500360096
:10306800384090000034a100304498001e009000c1
:103078000000e9008a80b90000804400e0b09000b8
:10308800efc060002841900000cfb300004061000d
:103098000140700020449800a848900080cfb300f9
:1030a80080c060003140b300214c98001e019000a0
:1030b8000201e8008a91b90082804400d1b89000ea
:1030c80068699000616c9800c808de007869900013
:1030d800716c9800b840900000c060000004a00027
:1030e80030449800284890008041b300204c980054
:1030f800420037001e0090000000e000240032006b
:10310800b91890001e0090008100e900808f5000df
:103118001f003a00384090000034a1003044980065
:103128001e0090000000e9008a80b9000080440079
:10313800e0b09000efc060002841900000cfb300dd
:10314800004061000140700020449800a8489000a9
:1031580080cfb30080c06000214c9800e8689000e0
:103168008040eb00616c980078699000716c980061
:10317800b840900000c060000004a00030449800ef
:10318800284890008041b300204c98001b0037006d
:1031980039189000e10f500018003a0038409000ac
:1031a8000034a10030449800a840900000cfb3003c
:1031b80000c0600020449800a848900080cfb30069
:1031c80080c060003140b300214c9800e86890004e
:1031d8008040eb00616c980078699000716c9800f1
:1031e800b840900000c060000004a000304498007f
:1031f800284890008041b300204c98001e009000a1
:103208008a80b90000804400c0009100ffc06000bf
:10321800320020008208dd003848900067406000d6
:1032280001407000304c98001e0090008a80b90060
:1032380000804400d0009100ffc060004849900021
:1032480000ceb3000040610001407000404c98007f
:10325800484090000034a000404498002840900066
:103268000064a0002044980029189000e10f500045
:1032780041003a00384890000004a000304c980003
:10328800484890000064a000404c98001e00900040
:103298008a80b9000080440030089100a868900036
:1032a800206c98004800de00b8689000306c9800e8
:1032b8001e0090008a80b9000080440040089100f8
:1032c800c8689000406c98004800de00d8689000fc
:1032d800506c9800685090000040eb0060549800d3
:1032e8007850900010c1b3007054980008589000ae
:1032f80090c1b300005c98001858900030c0b3002b
:10330800105c98001e0090008a80b900008044007c
:1033180090089100ffc060006851900000ceb30093
:103328000040610001407000605498001e00900049
:103338008a80b9000080440040f091000004e00059
:10334800070032006840900080c0b30060449800d5
:103358007840900000c3b30070449800060037001e
:103368006840900040c0b3006044980078409000e6
:1033780000c3b300704498001e0090000000e800ed
:1033880010079800b91890001e009000808f500018
:103398003dfe3e0029189000e10f500005003a005c
:1033a800e01707001e0f600009007800760b070081
:1033b8001e0f60001e0078004f05be004f04be00bf
:0833c8000080fa00000006007d
:020000040000fa
:1033d0000800fa006000b800c0bf9f00d1bf9f0086
:1033e0000000eb00e0bf9f00eca00a00840f00008b
:1033f000f0bf9f000120210031ae8800a10720000e
:1034000041ae88007fb897000000e000090032005c
:103410007fb89700e60f5000060032007fb8970093
:10342000e10f5000030032007fb89700e70f500013
:103430002d003a0000202100a1072000c0bf9f00fe
:10344000d1bf9f007fb89700e60f500013003200f5
:10345000627c800050820a00020000000281fb00b2
:103460008001eb0001eb2000819ab9000110b80047
:10347000810042004fb99700dfb997000001410079
:1034800081814900c2bf9f00d3bf9f004fba970000
:10349000dfba970034ae880045ae88007fb8970049
:1034a000e70f50001e003a0098a00a00860f0000a7
:1034b000e0bf9f004fb99700dfb99700efb89700c2
:1034c0000202be00010378000603e9000300330096
:1034d0008582d1000482d300fbff3700c4bf9f0068
:1034e000d5bf9f000e0037007fb89700e50f500052
:1034f00005003a0000d0270001002000c0bf9f0057
:10350000d1bf9f00060037004fb99700dfb9970081
:103510000000eb00e00f5100e08f59000401320081
:103520004fb89700dfb8970070ae880081ae880072
:103530007fb89700e10f5000030032007fb897007a
:10354000e30f500053003a000000eb0084afab00e3
:10355000f7003200307c80006f006000e0bf9f0009
:10356000efb897008100e9000000eb00e78f500002
:10357000ef003e004fb89700dfb897006fb9970093
:103580008001eb0015f50700c0bf9f00d1bf9f0071
:10359000f00f2000880fb600e0bf9f006fb99700c2
:1035a000630151000000eb00510c2000810f51001d
:1035b000df003e006fb897004fb99700dfb9970062
:1035c0008000eb00809ab9000200b8008100420040
:1035d000c0bf9f00d1bf9f0098a00a008a0f0000c3
:1035e000e0bf9f00efb897000000eb00e38f5000b2
:1035f000cf003e006fb8970064001000e0bf9f004e
:103600004fb89700dfb897006fb997008001eb00c3
:10361000f2f4070010af880021af880064a00a0010
:103620008a0f0000e0bf9f00efb897008100e9001b
:103630000000eb00e78f5000bd003e004fb8970040
:10364000dfb897006fb997008001eb00e3f4070043
:10365000c0bf9f00d1bf9f00507c8000670060000a
:10366000e0bf9f00efb897008100e9000000eb0089
:10367000e78f5000ae003e004fb89700dfb89700cc
:103680006fb997008001eb00d4f40700c0bf9f0022
:10369000d1bf9f004fb99700dfb99700f2ae880005
:1036a00003af88004fb89700dfb897008180d10042
:1036b0000080d300c0bf9f00d1bf9f004fba9700ca
:1036c000dfba970094ae8800a5ae88004fb8970087
:1036d000dfb897008180d1000080d300c0bf9f0079
:1036e000d1bf9f004fb89700dfb89700d0ae8800d9
:1036f000e1ae8800876fab000f003200dca00a004b
:10370000860f0000e0bf9f004fb99700dfb9970018
:10371000efb897000202be00010378000603e9003b
:10372000030033008582d1000482d300fbff370001
:10373000c4bf9f00d5bf9f004fb89700dfb8970068
:10374000b0ae8800c1ae8800b0ae8000c1ae8000cf
:10375000f3f407000001be000000200001f8230080
:10376000aef7070050af880061af8800d0ae800090
:10377000e1ae8000eaf407000001be000000200076
:1037800001f82300a5f7070030af880041af88009b
:103790008e0fe20061003d008f0fab00050032008c
:1037a00032ae800043ae8000c2bf9f00d3bf9f00f7
:1037b0000400370054ae800065ae8000c4bf9f0097
:1037c000d5bf9f00707c80006f006000e0bf9f004d
:1037d000efb897008100e9000000eb00e78f500090
:1037e00053003e004fb89700dfb897006fb99700bd
:1037f0008001eb0079f40700c0bf9f00d1bf9f009c
:10380000f00f2000900fb600e0bf9f006fb9970047
:10381000630151000000eb00510c2000810f5100aa
:1038200043003e006fb897004fb99700dfb997008b
:103830008000eb00809ab9000200b80081004200cd
:10384000c0bf9f00d1bf9f0098a00a00920f000048
:10385000e0bf9f00efb897000000eb00e38f50003f
:1038600033003e006fb8970064001000e0bf9f0077
:103870004fb89700dfb897006fb997008001eb0051
:1038800056f4070090af8800a1af880064a00a003a
:10389000920f0000e0bf9f00efb897008100e900a1
:1038a0000000eb00e78f500021003e004fb897006a
:1038b000dfb897006fb997008001eb0047f407006d
:1038c000c0bf9f00d1bf9f00907c80006700600058
:1038d000e0bf9f00efb897008100e9000000eb0017
:1038e000e78f500012003e004fb89700dfb89700f6
:1038f0006fb997008001eb0038f40700c0bf9f004c
:10390000d1bf9f004fb89700dfb8970070af880015
:1039100081af88001000200005003700ee35ef0071
:10392000f035ef00f235ef00f435ef001000200025
:083930000080fa00000006000f
:020000040000fa
:103938000600fa00889fbe0000047800d1bf9f00ef
:1039480010002000b0bf9f000000eb00c0bf9f0028
:1039580028189000e10f500063003200030039007e
:10396800e20f50003d013a0082003700b8a89100ec
:103978005fb89700808f50000300360038a8910088
:10398800d0bf9f0006003700c8a891005fb8970015
:10399800808f500002003100c8a89100d1bf9f005d
:1039a80098b191005fb9970058a891008000eb008a
:1039b8000300010058a89100a05090008180fb00ee
:1039c800305090004800dd00008070001c0032007c
:1039d80058a89100a05890008180fb0030589000b2
:1039e8004800dd00008070001500320058a89100e2
:1039f800104078000028a3001100320058a8910058
:103a0800a05090008180fb00305090004800dd00fd
:103a180000807000dfb897000108780058a891006e
:103a2800a05890008180fb00305890004800dd00cd
:103a380000807000dfb897000108780000013700a7
:103a480058a89100a05090008180fb003050900051
:103a58004800dd00008070000d00320058a8910079
:103a6800104090000048a30009003a0058a89100af
:103a7800a05090008180fb00305090004800dd008d
:103a880000807000dfb8970001087800ec0037006c
:103a980058a89100a05890008180fb0030589000f1
:103aa8004800dd00808070000000eb00f00032006c
:103ab80058a89100904090000000eb000148a30036
:103ac800eb00320058a89100a05890008180fb00bc
:103ad800305890004800dd0000807000dfb8970083
:103ae80001087800d6003700cfb8970040032000bf
:103af8008088b90000004400e00891000000eb0055
:103b08000100e000da003200f8a8910058a89100fe
:103b1800010001000000eb00c0bf9f00b818900032
:103b28004fb89700808f5000c50036004003200032
:103b38004fb997008091b90082004400e1089100d4
:103b48004fb997008091b9000201440072099100b1
:103b580082087800cfb897008100e800c1bf9f00b5
:103b680038199000cfb89700810f5100f0ff3e0040
:103b7800b30037000000eb00c0bf9f00b8189000ea
:103b88004fb89700808f5000ad0036008004eb00de
:103b98004fb89700f400b90000004400d0b091007d
:103ba8005fb89700808f5000060036004fb8970026
:103bb800f400b9000000440050b09100d0bf9f004d
:103bc8000c0037004fb89700f400b900000044001b
:103bd800e0b091005fb89700808f50000500310079
:103be8004fb89700f400b9000000440060b091009d
:103bf800d0bf9f004fb89700f400b9000000440000
:103c0800b0b991005fb997004fb89700f400b900b8
:103c18000000440070b091008900780003000100a2
:103c28004fb89700f400b9000000440070b091004c
:103c3800a05090008180fb00305090004800dd00cb
:103c4800008070003e0032004fb89700f400b900c1
:103c58000000440070b09100a05890008180fb00e3
:103c6800305890004800dd000080700034003200b9
:103c78004fb89700f400b9000000440070b09100fc
:103c8800104078000028a3002d0032004fb897009c
:103c9800f400b9000000440070b09100a0509000fa
:103ca8008180fb00305090004800dd0000807000eb
:103cb800dfb89700010878004fb89700f400b90002
:103cc8000000440070b09100a05890008180fb0073
:103cd800305890004800dd0000807000dfb8970081
:103ce800010878004fb89700f400b90000004400bc
:103cf80070b09100c04091008180fb00504091005d
:103d08004800dd0000807000dfb8970001087800e7
:103d18004fb89700f400b9000000440070b091005b
:103d2800e04091008180fb00704091004800dd0078
:103d380000807000dfb8970001087800390037006c
:103d48004fb89700f400b9000000440070b091002b
:103d5800a05090008180fb00305090004800dd00aa
:103d680000807000130032004fb89700f400b900cb
:103d78000000440070b09100104090000048a3007b
:103d88000c003a004fb89700f400b9000000440056
:103d980070b09100a05090008180fb0030509000de
:103da8004800dd0000807000dfb897000108780047
:103db8001c0037004fb89700f400b9000000440019
:103dc80070b09100a05890008180fb00305890009e
:103dd8004800dd0000807000220032004fb89700d4
:103de800f400b9000000440070b091001040900049
:103df8000048a3001d0032004fb89700f400b90036
:103e08000000440070b09100a05890008180fb0031
:103e1800305890004800dd0000807000dfb897003f
:103e2800010878004fb897000000e800c0bf9f0065
:103e3800b81890004fb89700808f500054ff3e008c
:103e48000800780073160700bfb8970001006000eb
:103e5800b0bf9f003fb89700050037000000eb0097
:103e6800030037000000eb00010037000000eb0002
:0c3e78004f04be000080fa0000000600ad
:020000040000fa
:103e84000614000084000000820000000382000089
:103e940000461000ffff000000ffff001503310083
:103ea400001e51007403870013000000038100000a
:103eb40000461000ffff000000ffff000b0f310061
:103ec400001e5100ad0e87001300000003810000a6
:103ed400004a1000ffff000000ffff004b06310006
:103ee400001e5100f4051f004e00000000010000f8
:103ef40000441000ffff000000ffff007c101300cf
:103f0400001e5100930d1f004e0000000001000030
:103f140000481000ffff380010ffff003f00f300cf
:103f2400011e510025001f004e00000006141e0053
:103f3400143614004e146600140500005a160000ce
:103f440018000000820000000300000000000000d0
:103f5400ffff000000ffff00000000000000000061
:103f64000000000000000000ea1600000c00000041
:103f740080000000fe160000060000008000000023
:103f8400001000003402000080000000ee14000065
:103f94006000000082000000030000000000000038
:103fa400000000000000000000000000000000000d
:103fb40000000000000000000000000000000000fd
:103fc40000000000000000000000000000000000ed
:103fd400880000000100000000300000001901000a
:103fe400400100000000000000000000000000008c
:103ff40000000000000000000000080000000000b5
:1040040000000000000000000000000000000000ac
:10401400000000000000000004170000040000007d
:1040240080000000f6160000080000008200000076
:10403400800000000054000089000000c016000049
:104044000e00000080000000ce1600000e000000ec
:10405400820000001e4f220048e04d00f846900008
:1040640045304b0006000000b016000010000000b0
:1040740082000000484fde0021fc41003a36220055
:104084004d0c4600a24d0700000000000817000078
:104094000400000082000000ec3101000000000078
:1040a4001a1600002000000080000000f615000031
:1040b400240000008200000002000300000200004f
:1040c4000300230078000000de07000000a4410084
:1040d4000000d200000000002fbf00000003000019
:1040e400010072005bffff00ee1200008c00000074
:1040f400800000008816000014000000800000000a
:10410400005000000a000000800000003a16000081
:1041140020000000820000000200030000020000f2
:104124000300bd00580000004427000000cd7100ca
:10413400000075000d000000a89b000000030000b3
:10414400040000007a1300008c00000080000000ce
:104154009c16000014000000800000000a500000bb
:104164000a0000008000000034120000ba000000c1
:1041740082000000000e1c000e380e00000011002a
:10418400110000000000000000000000000000001a
:10419400000000000000000000000000000001001a
:1041a4000000000000000200000000000000030006
:1041b40000000000000003000000000001000000f7
:1041c40000200000010001000021000001000200a5
:1041d400002200000100030000230000010004008d
:1041e4000024000001000500002500000100060075
:1041f400002600000100070000270000010008005d
:1042040000280000010009000029000001000a0044
:10421400002a000001000b00002b000001000c002c
:10422400002c000001000d00002d000001000e0014
:10423400002e000001000f00002f0000020000000b
:104244000030000002000100003100000200020002
:1042540000320000020003000033000002000400ea
:104264000034000002000500003500008c15000039
:104274003a000000820000002a0360000396030055
:10428400cc030200043804006e04a40004030000fc
:10429400000000000000000000000000000000001a
:1042a400000000000000000000000000000000000a
:1042b40000000000000000000000000000000000fa
:1042c4000000000000000000dc1600000e000000ea
:1042d40082000000880c98000ca80c0080000000ec
:1042e400005500008a000000c615000030000000e0
:1042f400800000008a1400006400000082000000b6
:104304000080020000000000000000000000000027
:1043140000000000008c5100f250ee003a085100f9
:104324000000000000000000000000000000000089
:1043340000000000800200000000000000000000f7
:104344000000000000000000dc501200509c4f00f0
:10435400d851000000000000000000000000000030
:1043640000000000008a1400b0140200008a140047
:10437400b0140200008a1400b0140200008a140071
:10438400b0140200000000004e1500003e000000c2
:10439400800000000c1700000400000082000000f0
:1043a40001000400000000001017000002000000db
:0843b400800000000000000081
:020000040000fa
:1043bc002000fa00881f780000047800100020000c
:1043cc00f0af9f000001eb0082b79f006000b800c7
:1043dc0090b79f00a1b79f00b0b79f00c1b79f00d7
:1043ec00d0b79f00e1b79f00f0b79f0081bf9f003f
:1043fc0090bf9f00a1bf9f00b0bf9f00c1bf9f0097
:10440c00d0bf9f00e1bf9f001870a000481890001b
:10441c0000ac990042149800720c980058a89100b6
:10442c00810220008880400020619000216098006b
:10443c00c808de003061900031609800c820900000
:10444c0041149800c810900068109000808f5000a4
:10445c00020031006812900044149800581090002b
:10446c000000e00002003a001000200050149800f8
:10447c00081090000000e00002003a00100020003c
:10448c0000149800b820900038309000808f5000b5
:10449c0075003200c820900068389000808f500062
:1044ac0071003200c83890004821900068389000a4
:1044bc00000051000100b80090b79f00a1b79f0009
:1044cc001fb19700afb19700d8389000f080100062
:1044dc000202be00010378000603e900030033006a
:1044ec008502d1000482d300fbff370094b79f00f4
:1044fc00a5b79f009830900038219000383090007c
:10450c00000051000100b800b0b79f00c1b79f0078
:10451c003fb19700cfb19700a8309000f080100009
:10452c000202be00010378000603e9000300330019
:10453c008502d1000482d300fbff3700b4b79f0083
:10454c00c5b79f001fb19700afb197003fb0970060
:10455c00cfb09700800f5100818f590004003600b6
:10456c003fb09700cfb0970090b79f00a1b79f00c6
:10457c00481890008000eb00f0b79f0081bf9f00af
:10458c0048b890008000eb00d0bf9f00e1bf9f00b7
:10459c003fb09700cfb09700e00f5000e08f58006d
:1045ac00210032005fb99700efb997001fb0970058
:1045bc00afb097000200b800d0b79f00e1b79f00e2
:1045cc003fb19700cfb197005fb29700efb2970061
:1045dc000500090042aad8008000eb00d0b79f006c
:1045ec00e1b79f005fb99700efb997007fb09700d4
:1045fc008fb897000200b80090bf9f00a1bf9f002a
:10460c003fb19700cfb197001fba9700afba970090
:10461c000500090042aad8008000eb0090bf9f0063
:10462c00a1bf9f002c0037000fb197004003200062
:10463c008091b9008200440071b990008001eb00b8
:10464c00d2b79f00e3b79f008fb097008088b90066
:10465c000000440070b890008000eb0090bf9f00f9
:10466c00a1bf9f001c0037000000eb0080b79f002b
:10467c00b81890000fb09700808f500016003600cd
:10468c00400320000fb197008091b90082004400d4
:10469c0071b990008001eb00d2b79f00e3b79f0087
:1046ac000fb197008091b9008200440071b990005d
:1046bc008001eb0092bf9f00a3bf9f008fb09700bb
:1046cc008100e80081b79f00381990008fb09700e7
:1046dc00810f5100ebff3e0028189000e10f5000b5
:1046ec000f00320003003900e20f50006e003a0058
:1046fc00160037005fb09700efb09700800078008d
:10470c000800780089fc07007faa9700040060006d
:10471c00f0af9f0010002000f0af9f006400370046
:10472c005fb09700efb09700800078000800780029
:10473c007efc0700ffaa970005006000f0af9f0009
:10474c0010002000f0af9f0059003700581b90005c
:10475c0046ac990058a89100c8a8910020c99000b7
:10476c0021c89800c808de0030c9900031c89800f4
:10477c005fb09700efb097008000780008007800d9
:10478c006afc0700ffa8970001006000f0af9f00d3
:10479c00686890000004e0004000320008189000a7
:1047ac001fb19700afb197008000eb0002005000e2
:1047bc0083805800f0b79f0081bf9f007fb09700a7
:1047cc008fb89700581190007fb097008fb8970062
:1047dc006102b8000500090042aad8008000eb0075
:1047ec00f0b79f0081bf9f001fb99700afb997002a
:1047fc005fb09700efb09700000051008180590026
:10480c00b0bf9f00c1bf9f003fb89700cfb89700c3
:10481c00e00f5000e08f580004003a001000200018
:10482c0001002000b0bf9f00c1bf9f007fb1970067
:10483c008fb997003fb89700cfb897006102b800c6
:10484c000500090042aad8008000eb00b0bf9f0011
:10485c00c1bf9f003fb89700cfb897008100d1002f
:10486c000080d300b0bf9f00c1bf9f003fb897002e
:10487c00cfb89700e00f5000e08f580004003a00ca
:10488c001000200001002000b0bf9f00c1bf9f009e
:10489c003fb89700cfb89700101c9800100020006c
:1048ac00f0af9f00020037000002eb00f4af9f0056
:1048bc007fa897004f0478000080fa0000000600e3
:020000040000fa
:1048cc000600fa00881f7800000478001000200011
:1048dc00c0bf9f000000eb00d0bf9f00e0bf9f0057
:1048ec0058a89100904090000174a10011409800cc
:1048fc00f8a8910058a891000100010038a8910077
:10490c00e0bf9f0058a89100a05090008180fb0050
:10491c00305090004800dd00008070001c00320018
:10492c0058a89100a05890008180fb00305890004e
:10493c004800dd00008070001500320058a891007e
:10494c00104078000028a3001100320058a89100f4
:10495c00a05090008180fb00305090004800dd009a
:10496c0000807000efb897000108780058a89100fb
:10497c00a05890008180fb00305890004800dd006a
:10498c0000807000efb8970001087800290037000c
:10499c0058a89100a05090008180fb0030509000ee
:1049ac004800dd00008070000d00320058a8910016
:1049bc00104090000048a30009003a0058a891004c
:1049cc00a05090008180fb00305090004800dd002a
:1049dc0000807000efb897000108780015003700d0
:1049ec0058a89100205990000281fb00b05890000b
:1049fc00c808dd00810071000000eb00d00032001f
:104a0c0058a89100904090000000eb000148a300d2
:104a1c00cb00320058a89100a05890008180fb0078
:104a2c00305890004800dd0000807000efb897000f
:104a3c000108780028189000e10f500004003200a3
:104a4c00b3003900e20f5000b8003a0023003700e1
:104a5c00dfb89700400320008088b90000004400b4
:104a6c00e00891000000eb000100e000b40032000f
:104a7c00f8a8910058a89100010001000000eb007b
:104a8c00d0bf9f00b81890005fb89700808f50007f
:104a9c009f003600400320005fb997008091b90059
:104aac0082004400e10891005fb997008091b90041
:104abc00020144007209910082087800dfb8970067
:104acc008100e800d1bf9f0038199000dfb8970033
:104adc00810f5100f0ff3e008d0037005fb897004a
:104aec00f400b9000000440070b0910090409000b8
:104afc000174a100114098000000eb00d0bf9f0092
:104b0c00b81890005fb89700808f50008000360076
:104b1c005fb89700f400b9000000440090b8910011
:104b2c005fb89700f400b9000000440070b0910029
:104b3c00010001005fb89700f400b90000004400c8
:104b4c0050b09100e0bf9f005fb89700f400b9002f
:104b5c000000440070b09100a05090008180fb00d8
:104b6c00305090004800dd000080700028003200ba
:104b7c005fb89700f400b9000000440070b09100d9
:104b8c00a05890008180fb00305890004800dd0058
:104b9c00008070001e0032005fb89700f400b9006e
:104bac000000440070b09100104078000028a30071
:104bbc00170032005fb89700f400b9000000440001
:104bcc0070b09100a05090008180fb00305090009c
:104bdc004800dd0000807000efb8970001087800f5
:104bec005fb89700f400b9000000440070b0910069
:104bfc00a05890008180fb00305890004800dd00e8
:104c0c0000807000efb89700010878003900370079
:104c1c005fb89700f400b9000000440070b0910038
:104c2c00a05090008180fb00305090004800dd00c7
:104c3c0000807000130032005fb89700f400b900d8
:104c4c000000440070b09100104090000048a30098
:104c5c000c003a005fb89700f400b9000000440063
:104c6c0070b09100a05090008180fb0030509000fb
:104c7c004800dd0000807000efb897000108780054
:104c8c001c0037005fb89700f400b9000000440026
:104c9c0070b09100a05890008180fb0030589000bb
:104cac004800dd0000807000220032005fb89700e1
:104cbc00f400b9000000440070b091001040900066
:104ccc000048a3001d0032005fb89700f400b90043
:104cdc000000440070b09100a05890008180fb004f
:104cec00305890004800dd0000807000efb897004d
:104cfc00010878005fb897000000e800d0bf9f0063
:104d0c00b81890005fb89700808f500080ff3e006d
:104d1c0008007800be120700cfb8970001006000b1
:104d2c00c0bf9f004fb89700050037000000eb0094
:104d3c00030037000000eb00010037000000eb001f
:0c4d4c004f0478000080fa000000060010
:020000040000fa
:104d58001800fa00889fbe008a1f78008104780036
:104d68001100200091b79f006011b800a2b79f0002
:104d7800b3b79f008000eb00c1b79f00d1b79f0079
:104d8800e1b79f00e1ef9f0082bf9f0093bf9f00a4
:104d9800ec01b90001562100810041009100780022
:104da800d1b79f0021002000e1b79f00818f5400f8
:104db80002003a004e35a80003003700e18f540086
:104dc80001003a004e15a8008000eb00c1b79f0013
:104dd8004fb19700dfb09700810f5100d700310025
:104de80000054000ec00b900c15521000104400055
:104df8000900e00003003a0010c0b300e0ef9f0094
:104e080036003700980078004fb097000000400047
:104e180000804000100078001000e0002d003d00e8
:104e2800980078004fb097000000400000804000d4
:104e38001000780010009000890f500022003a00fe
:104e4800980078004fb097000000400000804000b4
:104e58001000780040019000d00190009800780080
:104e68004fb097000000400000804000100078001c
:104e7800f00090006000900000004100818049002f
:104e880080bf9f0091bf9f00980078004fb09700a7
:104e980000004000008040001000780020029000d0
:104ea800b00290000fb997009fb9970010c0b300e7
:104eb800820f5200838f5a0001003d000040eb0032
:104ec800e0ef9f00050037000040eb00e0ef9f0097
:104ed800020037000040eb00e0ef9f006fe897000a
:104ee8000004e0008e003200980078004fb0970070
:104ef8000000400000804000100078007001400071
:104f08000a014100980078004fb097000000400067
:104f18000080400010007800e4004000980178000c
:104f28004fb097000000400000804100100078005a
:104f38001070a000120078007c815700470b070012
:104f480090b79f00980078004fb09700000040008d
:104f580000804000100078009fb0970001f0a70083
:104f68008100ea008100ea00cf08de0000010a00a3
:104f780010000000980078004fb097000000400033
:104f880000804000100078001070a1000028ab00dd
:104f98002a00320080aa800091aa800011a20a008b
:104fa8000008000000004100e080480080aa880056
:104fb80091aa880010002000a0bf9f000000eb000d
:104fc800b0bf9f00c0bf9f0082aa800093aa800044
:104fd800c2bf9f00b0bf9f003fb89700da14e3003c
:104fe80012003600644d21003fb8970000004000d1
:104ff800000042001000780020019000b0019000ed
:10500800cfb8970002814000e08149002200980053
:10501800330098003fb897000000e800b0bf9f0039
:105028003fb89700da14e300efff3e005035ef0079
:105038005235ef000028a9002fb897009800780093
:105048004fb097000000400000804000100078003a
:1050580020019000b001900082bf9f0093bf9f0085
:105068000fb997009fb99700980078004fb0970044
:10507800000040000080400010007800f000900020
:1050880060009000000051008180590080bf9f009f
:1050980091bf9f000fb997009fb9970098007800bb
:1050a8004fb09700000040000080400010007800da
:1050b800d00090004000900000005100818059000d
:1050c80080bf9f0091bf9f00980078004fb0970065
:1050d800000040000080400010007800f0009000c0
:1050e800600090000fb997009fb997000200400038
:1050f8008380480080bf9f0091bf9f009800780080
:105108004fb0970000004000008040001000780079
:105118000fb997009fb997002200980033009800b4
:105128004fb097000000e800c0b79f00cfb09700cd
:105138005fb09700808f50002dff39001fb0970097
:105148004f0578004f04be000080fa0000000600fa
:020000040000fa
:105158000400fa00889fbe0010002000c0bf9f0016
:105168008040eb00a1ff9f0068f0b700a0ff9f0000
:10517800b3c0b300f20621000349780081c0b30030
:10518800e4062100014a780022c2200052838800e8
:1051980042c0b30018072100024c78007470ef0079
:1051a8002ffa970023072100844978002ffc9700e5
:1051b80037072100884b78007670ef007570ef0094
:1051c800f3e92400c383880056002000d6838800b2
:1051d8007c30ef008406210014427800000262004f
:1051e8004922dd00e57080000590a100850272006b
:1051f800e570880052f0b700a5c0b30099052100fa
:10520800854c780087052100814b780004c2200076
:10521800a4828800b9052100824c78005e70ef00f6
:105228005c70ef005d70ef006070ef005f70ef0082
:1052380013838800268388006630ef002305210049
:105248009341780080816100c819dd00e470800016
:105258000480a10004827100e47088007ef0b70029
:1052680085f0b7008670ef0084f0b700e3c0200037
:10527800038488000244780077082100884b78006e
:105288008a70ef008870ef008970ef008c70ef0073
:105298008b70ef00f43f26007484880073002000b0
:1052a800838488000278200092848800e707210020
:1052b8009743780080836300c23bdd00e87080007c
:1052c8000820a10008847300e870880094f0b700f3
:1052d800e8c0b300b9092100884c7800a909210069
:1052e800814c780087c22000b7848800d809210043
:1052f800014c7800a070ef009e70ef009f70ef00e7
:10530800a270ef00a170ef00248588003385880023
:10531800428588004709210097437800808363000d
:10532800c23bdd00c87180000820a100088473001a
:10533800c8718800aaf0b70029c0b300180b210073
:10534800094c7800070b2100814b780007c1200029
:1053580067858800390b2100854c7800b670ef000e
:10536800b470ef00b570ef00b870ef00b770ef00e1
:10537800d4858800e3858800f2858800a70a210083
:105388009743780080836300833bdd00e8708000ea
:105398000870a10008847300e8708800c0f0b700a6
:1053a800d9c0b300780c2100094c7800670c2100a3
:1053b800814b780067c220001786880068c0b30058
:1053c800990c2100884c7800cc70ef00ca70ef006f
:1053d800cb70ef00ce70ef00cd70ef0084868800b0
:1053e80093868800a2868800020c2100124178006a
:1053f8000001610002014100c37180000310a10097
:1054080083017100c3718800d6f0b70006407800a8
:10541800ddf0b70081417800c20d21000349780012
:1054280060c12000c086880085437800f40d210003
:10543800074a7800e270ef00e070ef00e170ef00db
:10544800e470ef00e370ef00d6d0bf0000200a0040
:105458001c0e00004fb897004f04be000080fa00f1
:04546800000006003a
:020000040000fa
:10546c000400fa008002780011002000e1bf9f00c8
:10547c001504e000b6003200f5409000efcf50006c
:10548c0016003e0065499000f54090000281fb003b
:10549c008180fb008110dd0001007800d02bb7006b
:1054ac0035499000f54090000281fb008180fb00a3
:1054bc008110dd0001007800f02bb7002549900029
:1054cc00f54090000281fb008180fb008110dd0023
:1054dc0001007800202bb7001c00370075419000ac
:1054ec008000eb00ff4f51009a003e006549900090
:1054fc00f54090000281fb008180fb00f0805000a1
:10550c008110dd0001007800d22bb70035499000e6
:10551c00f54090000281fb008180fb00f080500080
:10552c008110dd0001007800f22bb70025499000b6
:10553c00f54090000281fb008180fb00f080500060
:10554c008110dd0001007800222bb700f54090009f
:10555c00e7cf500004003e00f540900081c04000b1
:10556c00e1ff9f0018003700f5409000efcf50008e
:10557c0005003e00f5409000e8c0500081c040009e
:10558c00e1ff9f0010003700f5409000f7cf50006e
:10559c0005003e00f5409000f0c0500081c0400076
:1055ac00e1ff9f0008003700754190008000eb0080
:1055bc00ff4f510067003e00f5409000f8c05000ce
:1055cc0081c04000e1ff9f00f540900001b1200038
:1055dc0091417800554a90006ff997000482fb00c6
:1055ec000281fb000221dd0082c87100914178002c
:1055fc00454a90006ff997000482fb000281fb0082
:10560c000201e8000221dd0082c87100f540900023
:10561c008180fb0002b82000828040001548900079
:10562c0080487800854890000104e0000b003200af
:10563c00e5409000e6cf500008003e000549900080
:10564c00e54090000281fb008180fb0081804000de
:10565c008110dd00010078000e2bb700e5409000b2
:10566c00e3cf50001d00320004003e00e1cf50009b
:10567c000e00320013003e0006003700e5cf50004c
:10568c00220032001b003900e6cf50002b003a00fc
:10569c00240037000417a800454890000004e000df
:1056ac002b0032000617a800290037000437a80089
:1056bc00454890000004e000250032000637a800a1
:1056cc00230037000457a800454890000004e00070
:1056dc001f0032000657a8001d0037000477a800f1
:1056ec00454890000004e000190032000677a8003d
:1056fc00170037000497a800454890000004e0000c
:10570c00130032000697a8001100370004b7a80058
:10571c00454890000004e0000d00320006b7a800d8
:10572c000b00370004d7a800454890000004e000a7
:10573c000700320006d7a8000500370004f7a800c0
:10574c00454890000004e0000100320006f7a80074
:10575c00efb89700010078000080fa000000060006
:020000040000fa
:10576c000400fa0011002000e1bf9f008000eb0054
:10577c00f1bf9f000000e000a20032002001900069
:10578c000200e0009f003200a000900011017800a0
:10579c00b000900081006100f1bf9f00c00090003c
:1057ac000100e00009003200c00090009101780077
:1057bc00d00090007fb9970081806100810051007a
:1057cc0001f0a7008100ea00f1bf9f00a8810a0048
:1057dc0010000000e38f50002400320005003c0054
:1057ec00e18f500009003200e28f500084003a0033
:1057fc0012003700e58f50003400320027003500ce
:10580c00e68f50007e003a003c00370060019000ab
:10581c00ffb89700810f5100020031001010a0005a
:10582c004100370010099000ffb89700810f51001c
:10583c003d0036001010a1003b00370060019000c5
:10584c00ffb89700810f5100020036001010a00025
:10585c003500370010099000ffb89700810f5100f8
:10586c00310031001010a1002f00370060019000b2
:10587c00ffb89700810f510002003a001010a000f1
:10588c002900370060019000ffb89700810f51008c
:10589c00250032001010a100230037006001900099
:1058ac00ffb89700810f5100020032001010a000c9
:1058bc001d00370060019000ffb89700810f510068
:1058cc0019003a001010a1001700370010099000c1
:1058dc00ffb89700810f5100060031006001900065
:1058ec00ffb89700810f5100020036001010a00085
:1058fc000d0037001010a1000b00370010099000ac
:10590c00ffb89700810f510004003e006001900029
:10591c00ffb89700810f5100020031001010a00059
:10592c00010037001010a1001018a300170032005e
:10593c0010017800e10061000104e00013003a005e
:10594c001000e00011003d00900090008100e80084
:10595c001100980010019000f0009000810f510090
:10596c00250039001000a000f000900011009800f4
:10597c00800890000100e0001f0032000008900039
:10598c0000000100e0bf9f001b00370010017800f1
:10599c00e10061000104e000020032001018a300d5
:1059ac00020032001000e000110035009000900061
:1059bc008100e8001100980010019000a0089000f0
:1059cc00810f51000c0039001000a100a0089000bc
:1059dc0011009800b00890000100e00006003200b1
:1059ec003008900000000100e0bf9f00020037006b
:1059fc008000eb0011009800efb897000100370011
:105a0c008000eb00010078000080fa000000060026
:020000040000fa
:105a1c001400fa0080bf9f0091bf9f00a2bf9f009f
:105a2c00b3bf9f00c4bf9f00d5bf9f00e6bf9f00c0
:105a3c00f7bf9f000000eb00e0b79f00f0b79f009e
:105a4c0000002700840fb60023003200a1092000bb
:105a5c000001eb008007200053f8200080497800fb
:105a6c008149780082497800e2072000207c800080
:105a7c00000161000200a0007105200060042000fc
:105a8c0043f82000804978008149780082497800e9
:105a9c00f2342c00eca10a00840f0000a8a00a002c
:105aac00840f000080cf5000050032007fb09700bb
:105abc008000e800f1b79f00820f5000f5ff360020
:105acc00ffb09700f0342c00808f5000020036009d
:105adc0040002000e0b79f00eca10a00840f0000fa
:105aec000fb897008180fb00808f50004b00320074
:105afc0084efab0049003a007fb897006300600068
:105b0c004800dd00f1cf2f00527c800082806000c5
:105b1c0081007000517c88003fb8970050200a002b
:105b2c00860f00004fb89700b0200a00880f0000c5
:105b3c005fb89700670060004400dd00f1f82f00ab
:105b4c00527c80008280600081007000517c880053
:105b5c006fb8970020200a008a0f00000fb9970039
:105b6c00a10920008007200053f82000804978000c
:105b7c008149780082497800eca10a00840f00006a
:105b8c00a8a00a00840f000080cf50002d00320026
:105b9c00e2072000207c8000000161000200a000d0
:105bac00710520006004200043f820008049780033
:105bbc008149780082497800f2342c00eca10a006b
:105bcc00840f0000a8a00a00840f000080cf5000b2
:105bdc00050032007fb097008000e800f1b79f000d
:105bec00820f5000f5ff3600eca10a00840f000074
:105bfc00a8a00a00840f000080cf500004003a00d7
:105c0c00ffb09700f0342c00808f50000d00360050
:105c1c0020002000e0b79f000a003700eca10a002a
:105c2c00840f00000fb897008180fb00808f50001c
:105c3c000400320084efab00020032008000200030
:105c4c00e0b79f0084efa80002022000f3342c0080
:105c5c00217c80000100610005003a007fb09700b4
:105c6c008000e800f1b79f00830f5000f8ff36006a
:105c7c0084afab0004003200ffb09700f0342c006e
:105c8c00808f50000200360000012000e0b79f001a
:105c9c006fb197000200e00004003a0033a00a0044
:105cac00840f000061001000010037006fb09700f6
:085cbc000080fa000000060060
:020000040000fa
:105cc4000200fa00881f7800000478000000eb004e
:105cd400e0bf9f00f0000a00180000008168210066
:105ce4004861900041649800c808de005861900043
:105cf4005164980001692100686190006164980012
:105d0400c808de00786190007164980001002500e5
:105d140008699000016c9800c808de0018699000ba
:105d2400116c98004100250028699000216c9800ae
:105d3400c808de0038699000316c980071978000c3
:105d44006871900061749800c808de007871900052
:105d540071749800a1b0800008799000017c9800cb
:105d6400c808de0018799000117c980081978000a3
:105d740028799000217c9800c808de0038799000ca
:105d8400317c980091b08000487190004174980073
:105d9400c808de005871900051749800b1af8000bb
:105da40048699000416c9800c808de00586990006a
:105db400516c9800c1af800068699000616c9800d4
:105dc400c808de0078699000716c9800d1af80003b
:105dd4000871900001749800c808de0018719000e2
:105de40011749800e1af800028719000217498002c
:105df400c808de003871900031749800e0bf9f003d
:105e0400c86890008180fb00586890004800dd005d
:105e140000807000efb89700810f50001500360025
:105e2400e35f2100826821006fb89700efb8970004
:105e3400c208dd00818041004200dd000000410015
:105e440031187800211078006fb897000000e8003e
:105e5400e0bf9f00c86890008180fb0058689000f4
:105e64004800dd0000807000efb89700810f5000fb
:105e7400edff3e000000eb00e0bf9f00e8689000eb
:105e84008180fb00786890004800dd00008070008d
:105e9400efb89700810f50001600360063602100b0
:105ea400826821006fb89700efb89700c208dd0040
:105eb400818041000080e8004200dd0000004100d4
:105ec40031187800211078006fb897000000e800be
:105ed400e0bf9f00e86890008180fb007868900034
:105ee4004800dd0000807000efb89700810f50007b
:105ef400ecff3e00202f21000a050700b0b080000f
:105f0400e8789000607c98004800de00f878900003
:105f1400707c9800c0b08000c8789000407c9800e5
:105f24004800de00d8789000507c980010002000d3
:0c5f34004f0478000080fa000000060016
:020000040000fa
:105f40000200fa00881f7800000478000000eb00cf
:105f5000e0bf9f00f0000a0018000000c1692100a6
:105f60004861900041649800c808de0058619000c4
:105f700051649800416a2100686190006164980052
:105f8000c808de007861900071649800a1002500c7
:105f900008699000016c9800c808de00186990003c
:105fa000116c9800e100250028699000216c980090
:105fb000c808de0038699000316c9800d19b8000e1
:105fc0006871900061749800c808de0078719000d4
:105fd00071749800c1b2800008799000017c98002b
:105fe000c808de0018799000117c9800e19b8000c1
:105ff00028799000217c9800c808de00387990004c
:10600000317c9800b1b280004871900041749800d2
:10601000c808de005871900051749800d1b180001a
:1060200048699000416c9800c808de0058699000eb
:10603000516c9800e1b1800068699000616c980033
:10604000c808de0078699000716c9800f1b180009a
:106050000871900001749800c808de001871900063
:106060001174980001b2800028719000217498008a
:10607000c808de003871900031749800e0bf9f00be
:10608000c86890008180fb00586890004800dd00df
:1060900000807000efb89700810f500015003600a7
:1060a00023642100c26921006fb89700efb8970000
:1060b000c208dd00818041004200dd000000410097
:1060c00031187800211078006fb897000000e800c0
:1060d000e0bf9f00c86890008180fb005868900076
:1060e0004800dd0000807000efb89700810f50007d
:1060f000edff3e000000eb00e0bf9f00e86890006d
:106100008180fb00786890004800dd00008070000e
:10611000efb89700810f500016003600a3642100ed
:10612000c26921006fb89700efb89700c208dd0080
:10613000818041000080e8004200dd000000410055
:1061400031187800211078006fb897000000e8003f
:10615000e0bf9f00e86890008180fb0078689000b5
:106160004800dd0000807000efb89700810f5000fc
:10617000ecff3e00e0372100fc0407001824a000db
:10618000100020004f0478000080fa000000060094
:020000040000fa
:106190000600fa00889fbe008a9fbe008004780037
:1061a0001000200090bf9f000000eb00a0bf9f00e8
:1061b000b0bf9f00a0bf9f00b91890002fb89700f4
:1061c000808f50007f0036004a0320000b20200003
:1061d0002fb897008a80b9000080440060009100c9
:1061e0000000e90000004000c16d21000080400077
:1061f000100478009880fb00184090004800dd00f3
:10620000008070000b006000b0bf9f002fb89700a7
:106210008a80b900008044006000910001b68000cf
:1062200012b6800023b6800034b6800045b68000e8
:1062300056b6800067b68000d20e07009fb8970060
:106240000100600090bf9f003fb897006000b3005e
:10625000f0000a00180000002fb897008a80b900eb
:106260000080440000089100674060003100200079
:106270000100dd0071ccb30098c0600000cc70005c
:10628000284090000040eb0020449800b840900067
:10629000304498002fb997008a91b9008280440059
:1062a000b1009100f13fb2002841900021449800d4
:1062b000c808de00b8419000c2cfb30002c161003f
:1062c00081407100314498002fb997008a91b9003c
:1062d00082804400a108910048499000414c9800f8
:1062e000c808de0058499000514c98002fb997001b
:1062f0008a91b90082804400d108910068419000e1
:1063000061449800c808de0078419000714498000c
:10631000c840900040449800d840900050449800f5
:1063200088489000004c980098489000104c9800c5
:106330002fb897008a80b9000080440060b19000b7
:106340006f4161008848900000cfb30080c06000ba
:1063500082c07000014c98002fb997008a91b90053
:1063600082804400e1b09000efc0600018499000c6
:106370000040610001407000104c98002fb8970059
:106380008a80b90000804400f0009100efc06000f6
:10639000420020008208dd00084890006f40600045
:1063a00001407000004c98002fb897000000e800f2
:1063b000a0bf9f00b91890002fb89700808f5000a1
:1063c00083ff3e001fb897004f05be004f04be007c
:0863d0000080fa000000060045
:020000040000fa
:1063d8000600fa00889fbe008a9fbe008c9fbe0000
:1063e8008000eb00f1b79f0012c0b30082f79f0056
:1063f80091bf9f00110020001088a3007e0032008a
:10640800210020001018a3007b0032001028a300f0
:10641800790032008000eb00f1b79f00b0189000bf
:106428007fb19700828f50006a003600a161210079
:10643800e48240000182e8008003eb0016c0b3004c
:106448000044eb007fb197004311dd00028140005a
:106458001204e000170032007fb197004311dd00fd
:1064680002814000124190000204e0001100320055
:106478007fb197004311dd00028142006055b800ea
:106488000a89be007fb197004311dd000201420076
:10649800070978007fb197004311dd0002814000b1
:1064a800074978007fb197004311dd000281400061
:1064b80017419800ffb19700c319dd000381400020
:1064c80012019000830142008209e800e70f5100a1
:1064d80017003e007fb197004311dd0002814000a4
:1064e800064978007fb197004311dd000281400022
:1064f800184198007fb197004311dd008281400068
:1065080023069000b3069000ffb59700fe81450072
:106518008381410083014000930178000281420099
:106528000c854100e0854e000a89be00180037003e
:106538007fb197004311dd0082814000230690005f
:10654800b3069000cd6ddd004366de000c86750055
:10655800c36ede00028142000c89be007fb1970045
:106568004311dd0002814000164198007fb1970079
:10657800ffb19700c319dd00838140002306900016
:10658800b3069000f411b900020140003cb1990033
:106598000ff19700ffb19700c319dd008381400018
:1065a800934190000281fb00030161000201ea00af
:1065b8004f11de0082f79f007fb197000201e800cb
:1065c800f2b79f0030199000ffb19700830f510078
:1065d8009cff3e000ff097000004e000030032002b
:1065e8001000200090bf9f0002003700200020000c
:1065f80090bf9f009fb89700010078004f06be002b
:106608004f05be004f04be000080fa0000000600df
:020000040000fa
:106618000600fa00889fbe008a9fbe008c9fbe00bd
:1066280010002000f0b79f000000eb0080bf9f0023
:1066380090bf9f004e35ef000e17f8005a15f9006d
:1066480080bf9f000fb897000e17e3007100360057
:10665800eb012900ca55210069022900640445009c
:106668008883e900a0552100420620006803400005
:106678008001eb000fbe97008fb897008180400023
:1066880081804500ec66b9000c064500110e7800c3
:106698008fbe97008fb897008180400081804400aa
:1066a80011067800ec6ab900840078008100440083
:1066b8009c0878000fbe9700ec66b9008c804300f8
:1066c8008fba9700850878008fb897000fbe97009b
:1066d800ec66b9000c0640002c0690000c06e80099
:1066e80082e6b9008100e800ec0ab900840078006d
:1066f800810040008c0878000fbe9700ec66b90056
:106708008c0043006022b8008488be0093bf9f00bd
:106718000fbe9700ec66b9008c004000310690006f
:106728009fb89700810f5600330036000fbe9700c0
:10673800ec66b9008c004000110690009fb89700e5
:106748008180400081004600110678008fb89700cc
:10675800ec0ab9008400780081004000910690009e
:106768009fb89700818040008180460091007800a2
:10677800910090009fbe9700828ab900840078003b
:106788008d804000211698000fbe9700ec66b90076
:106798008c004000110690009fb89700818040004f
:1067a80081004600910078001170a1000fbe97008b
:1067b800ec66b9008c004000110690009fb8970065
:1067c8008180400081004600910078001100a100fe
:1067d8009fb897008100e80091bf9f000fbe970007
:1067e800ec66b9008c004000310690009fb8970015
:1067f800810f5600cdff3e008fb897008100e8005a
:1068080081bf9f008fb8970075b88000818f5200b4
:1068180098ff3e00680a0700ffb09700010060007b
:10682800f0b79f007fb097004f06be004f05be002f
:0c6838004f04be000080fa0000000600c3
:020000040000fa
:106844000400fa00881f780000047800100020007b
:10685400d0bf9f000000eb000800e0007d00320084
:10686400487893000004e00018003200c01b2000a8
:10687400080040000c0c07000080fb00e0bf9f00f4
:1068840018a091000000e00009003a006fb89700da
:106894000000a20000f0a7000000ea000000e900e8
:1068a4004f00de00ff000a00180000000700370058
:1068b4006fb8970000f0a7000000ea000000e900ac
:1068c4004f00de00ff000a00180000001800e0007e
:1068d40006003d001868a30004003a001838a3001d
:1068e40002003a001818a3001b003a009800780030
:1068f400618060000004e00005003a001000200000
:1069040001002000100498002104980004003700be
:1069140020002000010020001004980021049800a9
:106924001800900000004000e16c2100008040004d
:10693400900078000800780001000100d0bf9f009b
:106944005fb8970000f0a7000000ea000000ea002a
:106954004f00de003f00370018009000da16e30015
:1069640004003e00100020000100200010049800e4
:10697400210498001800900000004000e16c210000
:10698400808040000000eb001100e0003100320084
:106994001800900000004000e16c210000804000dd
:1069a400900078000800780001000100d0bf9f002b
:1069b4005fb89700e10f50000b003200030039006c
:1069c400e20f50001b003a001700370010002000af
:1069d4000100200010049800210498000000eb003e
:1069e400d0bf9f0019003700180090006101b80063
:1069f40012049800230498000000e8001004980092
:106a040018009000da16e30004003e002000200085
:106a140001002000100498002104980010002000b8
:106a2400d0bf9f000900370010002000d0bf9f0096
:106a34000600370010002000010020001004980018
:106a4400210498008000eb00d1bf9f001810a10022
:106a54005fb897004f0478000080fa000000060039
:020000040000fa
:106a64000a00fa00889fbe008a9fbe001100200021
:106a7400f1b79f008000eb0081bf9f0091bf9f0092
:106a8400a1bf9f00b1bf9f0081bf9f00301990003c
:106a94008fb89700810f51006c0036004603200028
:106aa400c95821000800230037ff2f0005002800e3
:106ab400743821000a0024008b0020000fb99700cd
:106ac4008691b90082004000e1b09000a1bf9f0010
:106ad400afb897008100e9008180400081804400c4
:106ae40091007800e14190008381fb0071419000a6
:106af4004811dd000281710002017400e14190003f
:106b0400e24098004811de00f1419000f240980004
:106b1400814990008381fb00114990004811dd00f8
:106b24000281710007016100814990008248980048
:106b34004811de009149900092489800114190005c
:106b44000274a00092409800414190000234a000d9
:106b5400c24098001181fb00914190004711de0072
:106b64000e003200031880000381620005003a0021
:106b74001fb997008201e80093bf9f00840f510062
:106b8400f8ff36001fb99700840f510031003e0012
:106b9400031880000301650030003a000fb9970024
:106ba4008691b9000201400072f191000204e000f4
:106bb40003003200c2002000b2bf9f000a00370069
:106bc4000fb997008691b9000201400042f191008b
:106bd4000204e0000300320042002000b2bf9f0024
:106be40001003700bbbf9f00814990008381fb00f7
:106bf400114990004811dd0002817100bfb997006e
:106c04000301710081499000824898004811de0018
:106c140091499000924898009140900077810a0031
:106c2400010000007fb1970082806000f1b79f00ef
:106c34008fb897008100e80081bf9f003019900051
:106c44008fb89700810f51009cff3e007fb09700e2
:106c5400030037000000eb00010037000000eb00e8
:106c64004f05be004f04be000080fa00000006007d
:020000040000fa
:106c74000800fa00881f7800000478001000200043
:106c8400b0bf9f000000eb00c0bf9f00d0bf9f00bb
:106c9400e0bf9f001870a000686890000004e00046
:106ca40004003a0010002000b0bf9f003fb89700d6
:106cb4006c003700c820900008189000808f5000a6
:106cc4002800310058a89100904090000174a10060
:106cd400114098000000eb00c0bf9f00b81890005e
:106ce4004fb89700808f50001b0036004fb89700b4
:106cf400f400b9000000440070b09100904090008e
:106d04000174a100114098000800780058000700a1
:106d1400d0bf9f0018189000dfb897000080400093
:106d2400d0bf9f00dfb897000800780001f3070088
:106d3400bfb8970001006000b0bf9f004fb8970034
:106d44000000e800c0bf9f00b81890004fb897003b
:106d5400808f5000e5ff3e0020002000b0bf9f0060
:106d64003f003700c820900008189000808f500022
:106d740039003900482090004014980048109000d1
:106d8400d81090000080400040149800281890000b
:106d9400e20f500006003a003819900028209000b5
:106da4006102b8000500090042aad800e0bf9f00b4
:106db40098b191006fb9970058a891008000eb003a
:106dc4000300010058a89100904090000174a000b5
:106dd400114098000800780025000700d0bf9f00ec
:106de400dfb8970008007800d2f20700b0bf9f0018
:106df40028189000e20f500014003a000000eb0045
:106e0400c0bf9f00b81890004fb89700808f500003
:106e14000e0036004fb89700f400b900000044009b
:106e240070b09100904090000174a000114098004f
:106e34004fb897000000e800c0bf9f00b81890004a
:106e44004fb89700808f5000f2ff3e0010002000e2
:106e5400b0bf9f00020037000000eb00b0bf9f00ee
:106e64003fb897004f0478000080fa000000060045
:020000040000fa
:106e74000200fa0011002000f1bf9f00a01890004a
:106e8400e18f50003900320003003900e28f5000d6
:106e94006f003a0038003700d0a8910021519000cb
:106ea4000281fb00b1509000c808dd008100710030
:106eb40018003200d0a89100215990000281fb00f3
:106ec400b1589000c808dd00810071001100320043
:106ed400d0a89100914078000128a30004003a0052
:106ee400d0a89100914090000148a30009003a0005
:106ef40050a89100a05090008180fb003050900079
:106f04004800dd000080700010007800f0bf9f0092
:106f14004d003700d0a89100a15990008381fb0057
:106f2400315990004811dd00028171008000eb00ae
:106f340048003200d0a89100114190008000eb007d
:106f44000248a3004300320050a89100a0589000ca
:106f54008180fb00305890004800dd000080700004
:106f640010007800f0bf9f003700370070089100d0
:106f7400f0bf9f0034003700f0b091002151900021
:106f84000281fb00b1509000c808dd00810071004f
:106f940018003200f0b09100215990000281fb00ea
:106fa400b1589000c808dd00810071001100320062
:106fb400f0b09100914078000128a30004003a0049
:106fc400f0b09100914090000148a30009003a00fc
:106fd40070b09100a05090008180fb003050900070
:106fe4004800dd000080700010007800f0bf9f00b2
:106ff40015003700f0b09100a15990008381fb0087
:10700400315990004811dd00028171008000eb00cd
:1070140010003200f0b09100114190008000eb00ac
:107024000248a3000b00320070b09100a0589000f9
:107034008180fb00305890004800dd000080700023
:1070440010007800f0bf9f00ffb8970001003700e0
:107054008000eb00010078000080fa0000000600c8
:020000040000fa
:107064000200fa0011002000f1bf9f009000900080
:10707400818040004223210081004100910078007a
:10708400300190000200e00010003a0061429000dc
:107094000482fb00f1419000c819dd0083017200f5
:1070a40020019000140020000221dd000281ea008a
:1070b40003016100e1419000e24098004811de00c4
:1070c400f1419000f24098000e00370061429000b8
:1070d4000482fb00f1419000c819dd0083017200b5
:1070e40020019000140020000221dd0002817100c3
:1070f400e1419000e24098004811de00f141900027
:10710400f240980040019000e10f51000f003a0056
:10711400214290000482fb00b1419000c819dd00b7
:107124008301720020019000140020000221dd0080
:1071340002817100a1419000a24098004811de0034
:10714400b1419000b24098000f00370021429000f6
:107154000482fb00b1419000c819dd008301720074
:1071640020019000140020000221dd000281ea00c9
:1071740003016100a1419000a24098004811de0083
:10718400b1419000b240980040019000e20f5100dc
:107194000f003a00014a90000482fb0091499000dc
:1071a400c819dd0083017200200190001400200042
:1071b4000221dd000281710081499000824898001b
:1071c4004811de0091499000924898000f00370062
:1071d400014a90000482fb0091499000c819dd0027
:1071e4008301720020019000140020000221dd00c0
:1071f4000281ea00030161008149900082489800fd
:107204004811de0091499000924898001182fb00d9
:1072140091419000c819dd008301720020019000a3
:10722400100020000201dd000281ea000301610078
:10723400f0020a0011000000f0bf9f007fb8970021
:087244000080fa0000000600c2
:020000040000fa
:10724c0010f0a6002d00370020149000401590007f
:10725c008608c3008608c1001201c100301b9000d3
:10726c000600c8001a039000260598000a03900037
:10727c00160598001001900010d0a7005001900046
:10728c0092007800502990000109780010119000ac
:10729c0092801000201990008208dd0030149000bc
:1072ac00010d78008688c3008688c1008688c100dd
:1072bc001281c100401b90000680c8000000cb006a
:1072cc000400cd00402390001620e6000602780052
:1072dc005023900016a0e60006027800100c9000d7
:1072ec00040c7800401590000a03900016059800d5
:1072fc00040d78008c39040000000000100190008f
:10730c00920078005029900001097800a038900074
:10731c00303890000100010000000600801f78004a
:10732c00401090000018eb000008eb004f007800b4
:10733c00801f7800501090000018eb000018eb0034
:10734c000008eb004f00780000000600801f78005a
:10735c00811f7800501090000118780001187800f7
:10736c0001087800cf0078004f007800801f78006b
:10737c00821f7800401090000218780002087800f4
:10738c004f0178004f0078000000060010f0a600b6
:10739c001a0037001001900010d0a7005001900087
:1073ac00920078005029900001097800101190008b
:1073bc0092801000201990008208dd00701b900054
:1073cc0060199000010278001301c1000200c8008e
:1073dc000400cd00402390001620e6000602780041
:1073ec005023900016a0e60006027800100c9000c6
:1073fc00040c78000c3a040000000000100190000e
:10740c0092007800502990000109780000000600d5
:10741c0010f0a6004f00370020149000401590008b
:10742c008608c3008608c1001201c100301b900001
:10743c000600c8001a039000260598000a03900065
:10744c001605980010019000920078004001900001
:10745c0081001100101190009280100020199000f2
:10746c008208dd0030149000010d78008688c3007e
:10747c008688c1008688c1001281c100401b900023
:10748c000680c8000000cb000400cd004023900013
:10749c001620e600060278005023900016a0e600a5
:1074ac0006027800100c9000040c780080119000fb
:1074bc0083014200500c9000030c7800c0399000fe
:1074cc008301420020849000030c7800d039900096
:1074dc008301420030849000030c7800419bde0055
:1074ec00703c900008054300108490000a0c780052
:1074fc00c039900083014200419bde00603c90004b
:10750c0008054300008490000a0c7800801190005c
:10751c0083014200419bde00302c900008054300a3
:10752c00202c90000a0c780041a3de00102c900057
:10753c0008054300002c90000a0c780040159000c0
:10754c000a03900016059800040d7800b43a040064
:10755c00000000001001900092007800000006006e
:10756c00801f7800401090000018eb000008eb0022
:10757c004f007800801f7800501090000018eb002e
:10758c000018eb000008eb004f007800000006002c
:10759c00801f7800811f780050109000011878002f
:1075ac000118780001087800cf0078004f007800af
:1075bc00801f7800821f780040109000021878001d
:1075cc00020878004f0178004f0078000000060098
:020000040000fa
:1075dc000800fa0010002000c0bf9f000000eb0064
:1075ec00d0bf9f00e0bf9f00f0bf9f00200cf800b1
:1075fc004610f9000e0cf8003c10f900280cf800ad
:10760c003e10f900100cf8004010f900260cf800a0
:10761c004210f900160cf8004a10f900e0bf9f0068
:10762c00b18180006fb89700808f50002c0036001d
:10763c00000021008001eb00efb89700fe804000b5
:10764c008180400081004000110178006fba9700e2
:10765c00f622b9008400400091889000810f5100ff
:10766c0006003100efb89700fe804000818040009a
:10767c0081004000830878000a003700efb89700bb
:10768c00fe804000818040008100400011027800a3
:10769c006fb99700f611b9000201400012899000f1
:1076ac0082085200efb89700fe80400081804000b5
:1076bc008100400011017800ffb897008100410063
:1076cc00f1bf9f00efb897008100e800e1bf9f0079
:1076dc00b2818000efb89700810f5100d6ff3e00b9
:1076ec007fb897000000e00002003d000000eb00b6
:1076fc00f0bf9f007fb89700208288005fb897008a
:10770c00cfb8970001006000c0bf9f001e000700ab
:10771c00cfb8970001006000c0bf9f00000021009f
:10772c0045fc0700cfb8970001006000c0bf9f0068
:10773c0010808000e30f5000030036002080800092
:10774c00e30f500003003e0010808000e50f500056
:10775c0008003a00d08e8000a06090008180fb0071
:10776c00306090004800dd000080700070a388003d
:10777c000200370067f4a9004ff4a9004fb8970036
:08778c000080fa000000060075
:020000040000fa
:107794000400fa0010002000e0bf9f000000eb008e
:1077a400f0bf9f0010808000e50f500002003200ff
:1077b4006fb897005b003700e1818000f0818000a2
:1077c40000805000f0bf9f007fb89700e80f400092
:1077d40007003d00fe16ed0081f32f00810f5000dd
:1077e40001003d0001007800f0b78800090037006f
:1077f4007fb89700e80f500006003400fe16ec0036
:10780400810c2000810f5000010034000100780039
:10781400f0b78800708f8000f1b78000006190009d
:1078240001609800c808de001061900011609800a3
:10783400e18180000082800000805000f0bf9f0042
:107844007fb89700e80f400007003d000017ed00e7
:1078540081f32f00810f500001003d0001007800ea
:1078640000b88800090037007fb89700e80f50007f
:10787400060034000017ec00810c2000810f50003a
:10788400010034000100780000b88800708f800087
:1078940001b8800000f9900001f89800c808de00e3
:1078a40010f9900011f89800e181800010828000a6
:1078b40000805000f0bf9f007fb89700e80f4000a1
:1078c40007003d000217ed0081f32f00810f5000e7
:1078d40001003d000100780010b88800090037005d
:1078e4007fb89700e80f5000060034000217ec0040
:1078f400810c2000810f5000010034000100780049
:1079040010b88800708f800011b8800020f99000b2
:1079140021f89800c808de0030f9900031f898008a
:0c7924006fb897000080fa000000060019
:020000040000fa
:107930000600fa00881f780011002000c1bf9f00d8
:107940008000eb00d1bf9f00e1bf9f00d1bf9f002f
:1079500030199000dfb89700810f51004f003600ba
:1079600043032000c75821000600230035ff2f00e5
:1079700004c8b3005fb997008391b900820040004a
:10798000e1b09000e1bf9f00efb897008100e900ef
:107990008180400081804300910078006144900024
:1079a0000884fb00714190004811dd000201740061
:1079b0000201730061449000e24098004811de002b
:1079c00071449000f2409800014c90000884fb0044
:1079d000114990004811dd000201740005016100a9
:1079e000014c9000824898004811de00114c900034
:1079f000924898001184fb00114190004811dd006d
:107a00000201740002f0a100f0020a00110000005f
:107a10005fb997008391b9000201400072b99000ec
:107a200041649000c26098004811de0051649000eb
:107a3000d2609800414490000884fb0051419000be
:107a40004811dd00020174000230a00041449000a2
:107a5000c24098004811de0051449000d240980086
:107a60009140900084c060008180fb008100e900ab
:107a7000cf08de004fb9970082806000c1bf9f0031
:107a8000dfb897008100e800d1bf9f003019900057
:107a9000dfb89700810f5100b6ff3e00e0c09300b1
:107aa0000104e00005003200601cb000dd030700a7
:107ab000cfb8970001006000c0bf9f004fb897008b
:0c7ac0004f0478000080fa00000006006f
:020000040000fa
:107acc000400fa00889fbe0000047800100020001b
:107adc00c0bf9f008004eb00d9bf9f000800780056
:107aec00f4040700cfb8970001006000c0bf9f00ee
:107afc000800780055ec0700cfb897000100600033
:107b0c00c0bf9f007c010700cfb897000100600048
:107b1c00c0bf9f00600d20000800400050f6070019
:107b2c00cfb8970001006000c0bf9f002005200067
:107b3c00080040004af60700cfb89700010060002b
:107b4c00c0bf9f00800620000800400044f60700dc
:107b5c00cfb8970001006000c0bf9f00d9bf9f0045
:107b6c00b81890005fb89700808f50000f00360057
:107b7c005fb89700f600b900e007b00000004400c1
:107b8c0037f60700cfb8970001006000c0bf9f0018
:107b9c005fb897000000e800d0bf9f00b8189000b5
:107bac005fb89700808f5000f1ff3e00080078000e
:107bbc0081070700cfb8970001006000c0bf9f008d
:107bcc0058a89100904090000174a10011409800b9
:107bdc0028189000e20f500015003a000000eb004e
:107bec00d0bf9f00b81890005fb89700808f5000ee
:107bfc00100036005fb89700f400b9000000440094
:107c0c0070b09100904090000174a1001140980058
:107c1c005fb897000000e800d0bf9f00b818900034
:107c2c005fb89700808f5000f2ff3e0001003700d4
:107c3c002818900018f0a10010002000010020006e
:107c4c0010049800210498004fb897004f04be0010
:087c5c000080fa0000000600a0
:020000040000fa
:107c64001400fa00889fbe00d0bf9f000104780072
:107c74008204780010002000c0b79f000000eb00d1
:107c8400d0b79f00e0b79f006000b800f0b79f0036
:107c940081bf9f0090bf9f00a1bf9f00b0bf9f0006
:107ca400c1bf9f005fb897000000e00003003a00e6
:107cb400800ceb00b91478004a0037001800be00ad
:107cc400f0b79f0081bf9f0021088000d1b79f00bb
:107cd4005fb8970000000100cfb09700010060007a
:107ce400c0b79f0020088000e0b79f001801be00c5
:107cf4007fb097008fb89700000051008180590031
:107d040090bf9f00a1bf9f001fb89700afb8970016
:107d1400e00f5000e08f580004003200e10f5000e3
:107d2400e08f580016003a0007003700efb09700c4
:107d34005fb09700008050008000eb00b0bf9f0050
:107d4400c1bf9f00230037005fb09700f17022008d
:107d5400008050008000eb00b0bf9f00c1bf9f00b7
:107d64006fb197003fb89700cfb89700000041006b
:107d7400e0804800b0bf9f00c1bf9f0015003700de
:107d84001fb99700afb99700f07022000011b80036
:107d9400b2bf9f00c3bf9f003fb99700cfb9970000
:107da400dfb097000100500000005100e08059004e
:107db400b0bf9f00c1bf9f006fb197003fb897004d
:107dc400cfb8970000004100e0804800b0bf9f009a
:107dd400c1bf9f003fb89700cfb89700808cbe000a
:107de4004fb097004f04be000080fa000000060068
:020000040000fa
:107df4000200fa00889fbe0010002000d0bf9f0040
:107e04006087880070878800e100200081878800ef
:107e1400f100200091878800f570ef00f6f0b700bc
:107e2400f7f0b700f470ef0005f42100c58788006f
:107e3400fa30ef00820c2000f2878800e287880085
:107e4400042c210004888800f980400011888800ef
:107e540021888800031e2000338888000a31ef003f
:107e6400360020004688880006898800108988002a
:107e7400a600200026898800b600200036898800e4
:107e84002971ef002af1b7002bf1b7002871ef0038
:107e940065898800077d2000778988009289880099
:107ea40082898800a4898800b1898800c1898800f2
:107eb400d38988003e31ef0076002000e6898800ef
:107ec40048002000a88a8800b08a88006900200041
:107ed400c98a880059002000d98a88005d71ef00a2
:107ee4005ef1b7005ff1b7005c71ef00058b8800ad
:107ef400178b8800328b8800228b8800448b880083
:107f0400518b8800618b8800738b8800988b880064
:107f1400868b880028002000488c8800508c8800bc
:107f2400c8002000688c8800d8002000788c880065
:107f34009171ef0092f1b70093f1b7009071ef00e7
:107f4400a58c8800b78c8800d28c8800c28c8800ed
:107f5400e48c8800f18c8800018d8800138d8800e2
:107f6400308d8800268d88005fb897004f04be00ce
:087f74000080fa000000060085
:020000040000fa
:107f7c000a00fa00881f780011002000a1bf9f00a2
:107f8c008000eb00b1bf9f0081ff9f00d1bf9f001d
:107f9c00e1bf9f00b1bf9f0030199000bfb89700a0
:107fac00810f51005000360043032000c4582100bb
:107fbc000500230007002200060021003fb99700ae
:107fcc008391b90082004000e1b09000d1bf9f00c6
:107fdc00dfb897008100e9008180400081004200f9
:107fec00910078003fb997008391b90002014000dd
:107ffc0072f1910082ff9f000ff9970099880a0097
:10800c00100000000884ea000281fb0002016400f9
:10801c000201ea004f11de0082ff9f000ff997006a
:10802c000204e00002003200e5bf9f0009003700a7
:10803c003fb997008391b9000201400042f19100d1
:10804c000204e00002003200e6bf9f00010037008e
:10805c00e7bf9f00414190000234a000c24098004d
:10806c00614190000281fb00714490004844dd00a6
:10807c00080471006fb997000281ea0008016100e1
:10808c0061449000e24098004811de007144900079
:10809c00f2409800614190000281fb00f140900099
:1080ac00c808dd00810071006fb997008100610084
:1080bc0001f0a7008100ea008100e900cf08de0092
:1080cc002fb9970082806000a1bf9f00bfb89700b6
:1080dc008100e800b1bf9f0030199000bfb8970035
:1080ec00810f5100b5ff3e002fb897004f04780068
:0880fc000080fa0000000600fc
:020000040000fa
:108104000400fa0010002000e0bf9f00bba00a009a
:10811400a00f0000e0ff9f00a16fa900a40fa90019
:108124006ff89700610060004b00dd00017d800066
:1081340001b0a10081007000017d880001eba9005d
:1081440001aba90000062000022bb70002eba90036
:1081540005eba90005cba900058ba8000070200041
:10816400042bb70003f82f002058800080806100a2
:108174000100a00021588800a100200090210a00dd
:10818400060b000007cba90007eba900f1ff2100b3
:1081940082b0200012896000098ba900096ba90034
:1081a400094ba900092ba900090ba90008eba90098
:1081b40008cba90001fc2f0080b0200010886000cb
:1081c40001302800515888000aeba9000a0ba900c5
:1081d4000a2ba9000c0ba9000c2ba900c1ff2f002e
:1081e400e2b020001289600031ff2f00e0b02000cf
:1081f4001088600000eca900000ca900002ca90064
:1082040000f02000022cb70002eca900020ca90027
:10821400022ca9008000eb0090210a00d80b00007a
:1082240090210a00d40b00000230200002007800e4
:10823400d62bb700b05e8000808061000100a000f2
:10824400b15e880001c0210001007800d62bb70080
:1082540002007800da2bb700d25e80000280610051
:108264000000a000d05e880001007800da2bb7007f
:0c8274006fb897000080fa0000000600c0
:020000040000fa
:108280000a00fa00881f780000047800e1bf9f0010
:1082900010002000a0bf9f000000eb00b0bf9f00b7
:1082a000c0bf9f00a0ff9f006fb89700b0bf9f00a6
:1082b0003fb897000000e0002a0032003fb8970066
:1082c0000000e900000040000000440010007800b9
:1082d00026f50700afb8970001006000a0bf9f001f
:1082e0002ff997003fb897000000e9000000400018
:1082f000000044001000780010007800e1006000e9
:108300000280fb00010070000000ea004f00de0068
:10831000a0ff9f003fb897000000e9000000400068
:108320000000440010007800100078006101600037
:108330003fb89700cfb897000281fb000000e9002a
:108340000010dd0000807000c0bf9f003fb89700a4
:108350000000e900b0bf9f003fb897000000e000b8
:10836000d6ff3a002ff8970000200a00ea16000016
:108370004fb8970060b78800f456e200170032004b
:108380002ff897000004e00014003a0070b7800056
:1083900081b780000001e80072b78800810f5000ab
:1083a00008003100f216e2000c00320090b78000a5
:1083b00000000100afb8970001006000a0bf9f005f
:1083c00006003700f016e20004003200ea16a800aa
:1083d000ea36a800f016f800ee16f900aff897009c
:1083e000406f2100014878002fb897004f047800b3
:0883f0000080fa000000060005
:020000040000fa
:1083f8000400fa00881f78000004780010002000ac
:10840800d0bf9f000000eb00e0bf9f001870a000e5
:1084180008007800ff040700dfb89700010060003b
:10842800d0bf9f0028189000e10f500010003200c4
:1084380003003900e20f500042003a0018003700ec
:1084480008007800cbfe0700dfb897000100600045
:10845800d0bf9f0058a89100904090000174a000e0
:108468001140980010002000d0bf9f00370037004f
:1084780008007800bffe0700dfb897000100600021
:10848800d0bf9f0058a89100904090000174a000b0
:108498001140980010002000d0bf9f002b0037002b
:1084a800686890000004e0001e003a0008007800a8
:1084b800b0fe0700dfb8970001006000d0bf9f0042
:1084c80058a89100904090000174a00011409800b5
:1084d8000000eb00e0bf9f00b81890006fb897004d
:1084e800808f5000140036006fb89700f400b90070
:1084f8000000440070b09100904090000174a0000a
:10850800114098006fb897000000e800e0bf9f0096
:10851800b81890006fb89700808f5000f2ff3e00a7
:10852800050037000800780092fe0700dfb89700c2
:1085380001006000d0bf9f0010002000d0bf9f0046
:10854800020037000000eb00d0bf9f005fb8970023
:0c8558004f0478000080fa0000000600cc
:020000040000fa
:108564001400fa00f0bf9f0010002000e0b79f0045
:10857400f0b79f00a0bf9f007fb89700c103200001
:10858400810f5000290032000d003e00fe0f500004
:108594001d00320003003e00f40f500043003a0077
:1085a4001600370081022000810f500019003200ac
:1085b400ea804000810f50003c003a001800370068
:1085c40001052000810f50001e00320004003e000f
:1085d400ea805000810f500034003a001600370042
:1085e400a1052000810f500019003200ea804000ec
:1085f400810f50002d003a00180037004001200080
:10860400b0bf9f0017003700e0012000b0bf9f00fb
:108614001400370080022000b0bf9f001100370013
:1086240020032000b0bf9f000e003700c0032000cd
:10863400b0bf9f000b00370060042000b0bf9f0054
:108644000800370000052000b0bf9f000500370078
:10865400a0052000b0bf9f000200370040062000a4
:10866400b0bf9f0020002000c0bf9f00100020006a
:10867400d0bf9f007fb097008fb897001fb99700b5
:10868400afb997003fba9700cfba97005fbb970086
:10869400efbb9700e0f40700efb097000100600023
:1086a400e0b79f006fb09700010037000000eb00b7
:0886b4000080fa00000006003e
:020000040000fa
:1086bc000600fa0011002000d1bf9f008000eb00e3
:1086cc00e1bf9f00e1bf9f0030199000efb8970009
:1086dc00810f51003a00360046032000c558210096
:1086ec00040023008041eb006fb997008691b9001c
:1086fc0082004000e1b09000f1bf9f00ffb89700ee
:10870c008100e90081804000818042009100780066
:10871c00e14390008783fb00714190004811dd001c
:10872c000281730002017200e1439000e240980064
:10873c004811de00f1439000f24098004161900036
:10874c00c360980051619000d3609800c1439000c1
:10875c008783fb00514190004811dd0002817300ba
:10876c000230a000c1439000c24098004811de00c6
:10877c00d1439000d2409800614190000281fb00ef
:10878c00f1409000c808dd00810071008480600019
:10879c008100ea00cf08de005fb99700828060009c
:1087ac00d1bf9f00efb897008100e800e1bf9f00a8
:1087bc0030199000efb89700810f5100caff3e00ae
:1087cc00e0c093000104e00005003200601cb00022
:1087dc0091000700dfb8970001006000d0bf9f0038
:0c87ec005fb897000080fa000000060053
:020000040000fa
:1087f8000400fa00881f78000004780010002000a8
:10880800d0bf9f000000eb00e0bf9f0058a8910078
:10881800904090000174a10011409800f8a89100c0
:1088280058a891000100010028189000e20f50009c
:108838001d003a000000eb00e0bf9f00b818900050
:108848006fb89700808f5000170036006fb89700f8
:10885800f400b9000000440070b09100904090000e
:108868000174a100114098006fb89700f400b90096
:108878000000440090b891006fb89700f400b90068
:108888000000440070b09100010001006fb897002b
:108898000000e800e0bf9f00b81890006fb897008c
:1088a800808f5000e9ff3e00080078006bf8070051
:1088b800dfb8970001006000d0bf9f005fb8970045
:1088c8000000e000010032001820a00028189000e5
:1088d800e10f500005003a00080078001003070077
:1088e800dfb8970001006000d0bf9f006102070059
:1088f800dfb8970001006000d0bf9f0018f0a0000b
:1089080010002000010020001004980021049800a5
:108918005fb897004f0478000080fa000000060056
:020000040000fa
:108928000400fa0012002000e2bf9f008000eb0064
:10893800f1bf9f00900090008180400043232100f8
:108948008180410091007800a00190000311dd00b2
:10895800f2bf9f00300090000000e0000d003a00d8
:10896800614190000281fb00714090004800dd00e9
:10897800000071007fb9970002007000614190000b
:10898800e04098004800de0071419000f0409800f7
:108998000d003700e14190008381fb007141900098
:1089a8004811dd00028171007fb897000080ea005d
:1089b8000200600061419000e04098004800de003d
:1089c80071419000f0409800e14190008381fb00e4
:1089d800714190004811dd0002817100c141900091
:1089e8008381fb00514090004800dd000080710049
:1089f800ffb89700020068000100600000f0a700bf
:108a08000000ea000000e9004f00de00e0bf9f0020
:0c8a18006fb897000080fa000000060014
:020000040000fa
:108a24000400fa0012002000e2bf9f008000eb0067
:108a3400f1bf9f00900090008180400043232100fb
:108a44008180410091007800a00190000311dd00b5
:108a5400f2bf9f00300090000000e0000e003a00da
:108a6400e14190008381fb00714190004811dd00d9
:108a7400028171007fb897000080ea000200600064
:108a840061419000e04098004800de007141900090
:108a9400f04098000c003700614190000281fb0017
:108aa400714090004800dd00000071007fb997001c
:108ab4000200700061419000e04098004800de0030
:108ac40071419000f0409800e14190008381fb00e7
:108ad400714190004811dd0002817100c141900094
:108ae4008381fb00514090004800dd00008071004c
:108af400ffb89700020068000100600000f0a700c2
:108b04000000ea000000e9004f00de00e0bf9f0023
:0c8b14006fb897000080fa000000060017
:020000040000fa
:108b20000200fa00881f7800000478000000eb00c3
:108b3000e0bf9f0028009000be16e30002003e0048
:108b40000000eb0020049800280090000000400086
:108b5000016b2100808040000000eb001100e0006c
:108b60002a0032002800900000004000016b210024
:108b700000804000900078000800780001000100ab
:108b8000e0bf9f006fb89700e10f50000400320073
:108b9000e20f50001a003a00e0bf9f001a003700b1
:108ba000280090000000e8002004980028009000b1
:108bb000be16e3000f00360020002000e0bf9f003b
:108bc00028009000e50f50000f003a002818900090
:108bd0000000e0000300320028189000e10f500070
:108be00009003a00280090000000e80020049800e6
:108bf0000500370010002000e0bf9f000200370092
:108c00000000eb00e0bf9f006fb897004f047800b2
:088c10000080fa0000000600dc
:020000040000fa
:108c18000200fa008000eb00f1bf9f001070a00076
:108c2800a0189000e28f500028003a00d0a89100c8
:108c3800a1c990008381fb0031c990004811dd0073
:108c4800028171008011900003014100a1c99000c8
:108c5800a2c898004811de00b1c99000b2c89800b7
:108c6800d00890008100e80051089800d0a8910031
:108c7800a1c990008381fb0031c990004811dd0033
:108c880002817100d0189000810f51000c0039004a
:108c9800d018900041a89900d0a8910040a8910050
:108ca80021c99000a0c898004800de0031c9900092
:108cb800b0c8980010002000f0bf9f000c003700db
:108cc80020002000f0bf9f0009003700d0a89100c5
:108cd80040a8910021c99000a0c898004800de0073
:108ce80031c99000b0c8980010002000f0bf9f0064
:0c8cf8007fb897000080fa000000060022
:020000040000fa
:108d04000c00fa00a0bf9f00b1bf9f00c2bf9f002c
:108d1400d3bf9f00e4bf9f00f5bf9f006fb89700cb
:108d2400630060004800dd00f1cf2f00927c8000da
:108d34008280600081007000917c8800f003200034
:108d4400afb897000080600050200a008e0f00002a
:108d54003fb89700b0200a00900f00004fb897006a
:108d6400670060004400dd00f1f82f00927c800071
:108d74008280600081007000917c88005fb8970059
:108d840020200a00920f00007fb897006100600065
:108d94004800dd00717c80000180a100810070002a
:108da400717c88007fb8970022800a0000000000d0
:108db4004f00dd00717c800001f0a1008100700093
:108dc400717c8800ffb897000000eb000128a30025
:108dd40004003200707c8000ff800a000000000064
:0c8de4000080fb000080fa000000060088
:020000040000fa
:108df0000200fa00881f7800000478000000eb00f1
:108e0000e0bf9f001800e00003003d0018e8a30049
:108e10000100320018d0a0008000eb0008007800ac
:108e2000a2030700e0bf9f006fb89700e10f50005a
:108e300003003200e20f50000b003a00060037003a
:108e40001850a0001870a100200020001800e000b9
:108e500009003500170037001850a1001870a00055
:108e600020002000130037001850a1001870a10046
:108e70000000eb000f0037002000200018d8a300ee
:108e80000c0032001818a3000a0032001828a300b2
:108e9000080032001838a30006003a001868a30042
:108ea00004003a001858a3000200320018d0a100b4
:108eb000100020004f0478000080fa000000060037
:020000040000fa
:108ec0000400fa00889fbe00800478001000200093
:108ed000000f7800bba00a00a00f000020479800f8
:108ee000a16fa900a52fa9002e409000610060008d
:108ef0004b00dd00017d800001b0a1008100700009
:108f0000017d88002be3a90061e3a90097e3a90094
:108f1000cde3a90003e4a90039e4a9006fe4a900a6
:108f2000a5e4a900af02b00068fd2f000f044400c3
:108f3000e04e210029000900305c7800a802b10051
:108f4000ea0407001e0f600059f0910088077800be
:108f50000004e00007003200c9b890000030200093
:108f60002049900021489800c808de003049900050
:108f7000314898001e0078004f04be000080fa00bf
:048f800000000600e7
:020000040000fa
:108f84000400fa00881f7800000478001000200014
:108f9400d0bf9f000000eb00e0bf9f0008007800f6
:108fa40062fa0700dfb8970001006000d0bf9f009d
:108fb40058a89100904090000174a10011409800bd
:108fc40028189000e20f500014003a000000eb0053
:108fd400e0bf9f00b81890006fb89700808f5000d2
:108fe4000e0036006fb89700f400b900000044008a
:108ff40070b09100904090000174a100114098005d
:109004006fb897000000e800e0bf9f00b818900018
:109014006fb89700808f5000f2ff3e0018f0a10057
:109024001000200001002000100498002104980082
:109034005fb897004f0478000080fa000000060033
:020000040000fa
:109044000200fa008000eb00f1bf9f00310098009d
:10905400010898001010a100a01890000100e00081
:1090640002003a001050a000050037001088a30049
:10907400020032001050a100010037001050a0007f
:10908400d0a89100114190000274a1009240980070
:10909400a0189000e28f500014003a008000eb000a
:1090a400f1bf9f00b01890007fb99700828f5000e5
:1090b4000e0036007fb99700f411b9008200400019
:1090c400f1b09100114190000274a1009240980007
:1090d400ffb897008100e800f1bf9f00b01890002e
:1090e4007fb99700828f5000f2ff3e001070a100fc
:1090f4001000a000100020000080fa00000006000c
:020000040000fa
:109104000400fa0010002000e0bf9f000000eb0004
:10911400f0bf9f000010a9000030a9000050a90072
:109124000070a8000090a9000110a9000130a90056
:1091340001d0a80001f0a90000d0a800110020006f
:10914400118088000430ef0021002000a1818800f4
:10915400f1412000d1818800c13b2000c1818800f9
:1091640041002000b1818800f0bf9f00b1818000e0
:109174007fb89700808f5000090036000001eb0093
:10918400e28188007fb897000000e800f0bf9f00ec
:10919400b18180007fb89700808f5000f8ff3e00b7
:1091a4004430ef004830ef004630ef004a30ef0023
:0c91b4006fb897000080fa000000060071
:020000040000fa
:1091c0000200fa0010002000f0bf9f0000102000f5
:1091d000904090000174a1001140980090409000d0
:1091e0000154a10011409800904090000144a1005a
:1091f00011409800904090000134a1001140980067
:10920000904090000124a1001140980090409000ef
:109210003140b300114098001074a100f1ccb300ac
:1092200010c860001024a1001014a100c0409000dc
:109230008040eb0041409800504190005140980020
:1092400080489000f1c0b300014898009048900019
:1092500071c2b30011489800f0f82f004008b60022
:109260000050a000004288000028a9002028a90082
:0c9270007fb897000080fa0000000600a4
:020000040000fa
:10927c000600fa0010002000d0bf9f000000eb0099
:10928c00e0bf9f00f0bf9f0001eba800f10f200092
:10929c0020b88000010060000060880020b88000c9
:1092ac004800dd000417b700f0bf9f0015c0b300e5
:1092bc0074a923000043eb0002608000ffb8970004
:1092cc006fb897008001e800e3bf9f00810f510049
:1092dc000600320085407800840f500001003600f3
:1092ec00864078000104e000f3ff3a006fb9970064
:1092fc000000eb0071a92300810f510006003e0015
:10930c0000f02f000a2bb60020b880000080fb0074
:10931c000a2bb7005fb897000080fa000000060027
:020000040000fa
:10932c000200fa00881f780010002000e0bf9f00a8
:10933c0008c82000616f2100914078008180fb00fb
:10934c00f7d6bf004800dd0000807000826f21005e
:10935c00124178000281fb00916f2100914078004e
:10936c00c808dd0081007100a36f210093417800d3
:10937c008381fb00b26f2100124178004811dd009f
:10938c0002817100c46f2100144278000482fb003a
:10939c00d36f210093417800c819dd00830172005e
:1093ac004c030700efb8970001006000e0bf9f007e
:1093bc00184090000074a100104498006fb89700fa
:0c93cc004f0478000080fa00000006004a
:020000040000fa
:1093d8000400fa00889fbe0010002000c0bf9f0054
:1093e8000000eb00d0bf9f0089f40700cfb89700ba
:1093f80001006000c0bf9f00b0010700cfb8970010
:1094080001006000c0bf9f004e15e2001600350045
:1094180009002800f85227000c57e2000500320026
:109428005fb897008000e800d1bf9f00880f500008
:10943800f9ff3600110020002000200044ee07004c
:10944800cfb8970001006000c0bf9f000000eb008c
:10945800d0bf9f0010c0b3000cf7b70071aa8000fe
:1094680001806400ecff32000000fe000000eb0009
:0c9478004f04be000080fa000000060057
:020000040000fa
:109484000200fa0010002000f0bf9f00000021003d
:109494008df90700ffb8970001006000f0bf9f003e
:1094a40022cea9001ecea90022aea9001eaea9009c
:1094b400a2030700ffb8970001006000f0bf9f00ff
:1094c40021c2b30060c2b30013020700ffb89700c3
:1094d40001006000f0bf9f0031c2b30050c2b3006e
:1094e4000d020700ffb8970001006000f0bf9f0065
:1094f4009c030700ffb8970001006000f0bf9f00c5
:10950400901a80004200de00a01a8800901a8000a1
:109514004200de00a01a88007fb897000080fa009d
:04952400000006003d
:020000040000fa
:109528000400fa008000eb00e1bf9f001200200059
:10953800f2bf9f00e1bf9f00b01890006fb997007d
:10954800828f50001700360044032000c36d2100ad
:109558006fb997008491b90082004000e100910042
:109568008100e900818040008180410091007800fd
:10957800314990000274a000b2489800114190004f
:109588000274a00092409800efb897008100e800ac
:10959800e1bf9f00b01890006fb99700828f50000c
:1095a800ebff3e0000c82000904090000174a0002e
:1095b800114098007fb897000080fa00000006006c
:020000040000fa
:1095c8000200fa0010002000f0bf9f00cbfe070049
:1095d800ffb8970001006000f0bf9f0003fa070082
:1095e800ffb8970001006000f0bf9f0078020700f5
:1095f800ffb8970001006000f0bf9f00d4ee07009d
:10960800ffb8970001006000f0bf9f005d000700f1
:10961800ffb8970001006000f0bf9f008de20700cf
:10962800ffb8970001006000f0bf9f0093ff07009c
:10963800ffb8970001006000f0bf9f0050020700cc
:10964800ffb8970001006000f0bf9f007fb8970047
:089658000080fa00000006008a
:020000040000fa
:109660004019900080a89100810f51001f00320026
:109670001070a0004019900080a89100810f510047
:109680000b00310000a99100d01090008100510022
:1096900001a8990000a99100c0189000810f510005
:1096a00013003100c018900001a899001000370085
:1096b0004019900080a89100810f51000c003600e5
:1096c00080a89100501190008100410001a89900ec
:1096d00000a99100c0189000810f510004003600cd
:1096e000c018900001a89900010037001070a10077
:0896f00020002000000006002c
:020000040000fa
:1096f8001000fa00f0bf9f001000200080bf9f00fc
:109708006fb897000000a000e0bf9f000000eb00ca
:10971800d0bf9f007fb9970001322000810f510010
:1097280016003e001000200090bf9f00ffb8970071
:10973800c208de00a1bf9f0021002000b1bf9f002a
:10974800c0bf9f006fb897000020a000e0bf9f0037
:109758001fb89700afb897003fb99700cfb99700e7
:109768005fba9700efba970064fd07008fb89700bb
:109778000100600080bf9f000fb897000080fa00ca
:0497880000000600d7
:020000040000fa
:10978c000200fa0010002000f0bf9f00f07c2000c7
:10979c0040808800703e2000308188002a30ef0025
:1097ac002830ef002c30ef00a0818000e20f500039
:1097bc000d003a002830ef00d00d200060818800a9
:1097cc00713e2000e18088002030ef001e30ef0059
:1097dc002230ef0013c0b300e202210003497800ed
:1097ec0080818800030037002e70ef00c03b200002
:1097fc0080818800f07c200090808800c03b200095
:10980c00a08088007fb897000080fa000000060056
:020000040000fa
:10981c000600fa0011002000d1bf9f008000eb0071
:10982c00e1bf9f00f1bf9f00e1bf9f003019900086
:10983c00efb89700810f510016003600440320004a
:10984c00c35821006fb997008491b9008200400081
:10985c00e1b09000f1bf9f00ffb897008100e900d4
:10986c00818040008180410091007800414190004e
:10987c000234a000c2409800efb897008100e800c5
:10988c00e1bf9f0030199000efb89700810f510095
:10989c00ecff3e005fb897000080fa000000060065
:020000040000fa
:1098ac000200fa0011c0b300e1ff9f00900090008d
:1098bc00818040004223210081004100910078000a
:1098cc00c14190008381fb00514190004811dd00a3
:1098dc0002817100a0009000130020008118dd00af
:1098ec008280600001f0a7008100ea008100ea009c
:1098fc00cf08de00e1ff9f0030009000830f500086
:10990c0008003a00eff897000180fb00008051003e
:10991c0000f0a7000000ea000000ea004f00de00a3
:10992c00e0ff9f006ff897000080fa00000006002f
:020000040000fa
:10993c000400fa00e0ff9f00f1ff9f0010002000e0
:10994c00e0bf9f007ff89700670060004400dd00d7
:10995c00f1f82f00024280008280600081007000cc
:10996c00014288000028a9006ff897006100600090
:10997c0000004000014180000110a1008100700036
:10998c000141880000102000904090000174a0005c
:10999c00114098001040900077800a0000000000f1
:1099ac00efb8970001006000e0bf9f006fb8970010
:0899bc000080fa000000060023
:020000040000fa
:1099c4000200fa00881f78000004780010002000cc
:1099d400e0bf9f00487893000004e00004003200d8
:1099e400c01b2000080040009df50700e0bf9f0059
:1099f40068c093000004e00004003200601c2000f2
:109a04000800400096f50700e0bf9f0068c093007f
:109a14000004e00006003200601c20000800400042
:109a2400fffb0700efb8970001006000e0bf9f0054
:109a34006fb897004f0478000080fa000000060019
:020000040000fa
:109a44000200fa0011002000f1bf9f001070a00076
:109a5400c010900050119000810041004110980006
:109a6400a01090008100e80021109800401190009f
:109a740080a89100810f51000c00360080a891004d
:109a840041109800d0a89100001db0002161900001
:109a9400a06098004800de0031619000b06098003a
:109aa40010002000f0bf9f000200370020002000bb
:109ab400f0bf9f007fb897000080fa000000060006
:020000040000fa
:109ac4000200fa00881f780018002000e8bf9f00f9
:109ad4008040eb000140780097ff0700efb8970043
:109ae40001006000e0bf9f008000eb0001007800ef
:109af40098ec0700efb8970001006000e0bf9f00fa
:109b04008000eb000800780092ec0700efb89700a3
:109b140001006000e0bf9f0021c0b300084078004e
:109b240085ff0700efb8970001006000e0bf9f00c9
:109b34006fb897004f0478000080fa000000060018
:020000040000fa
:109b44000200fa008000eb00f1bf9f001070a0003b
:109b540080089000100990008101e8000308980033
:109b6400828f500010003600900890008100e800b9
:109b740001089800e0c093000104e00007003200ef
:109b8400601cb00067fb0700f0bf9f000000eb0003
:109b9400ffb897000100e00006003200100020002a
:109ba400f0bf9f000200370020002000f0bf9f009c
:0c9bb4007fb897000080fa000000060057
:020000040000fa
:109bc0000200fa00881f78000004780010002000ce
:109bd000e0bf9f0008007800b8fa0700efb89700d0
:109be00001006000e0bf9f000800780037eb07002d
:109bf000efb8970001006000e0bf9f000000eb009d
:109c000030049800000c9800500c98002014980024
:109c10001810a1001870a1006fb8970000f0a700fd
:109c20000000ea000000ea004f00de004f04780068
:089c30000080fa0000000600ac
:020000040000fa
:109c38000600fa00f1bf9f0011002000d1bf9f006d
:109c48008000eb00e1bf9f00e1bf9f006fb9970064
:109c5800ffb89700810f51000f003100efb897004f
:109c6800818040008100400091007800a2652100b9
:109c78000b000900b21878008101b100efb8970015
:109c88008100e800e1bf9f006fb99700ffb8970017
:109c9800810f5100f1ff39005fb897000080fa008a
:049ca80000000600b2
:020000040000fa
:109cac000400fa00f1bf9f008000eb00e1bf9f00b1
:109cbc000000e000130032007fb9970053b8800019
:109ccc00828f51000f003600ffb897008180400052
:109cdc0082702100010141008000eb001200e000c5
:109cec0008003200ffb8970081804000827021008c
:109cfc00810041009100780001000100e0bf9f004d
:109d0c00efb89700010078000080fa000000060010
:020000040000fa
:109d1c000600fa00e0ff9f00f1ff9f000000eb003f
:109d2c00d0bf9f00c0ff9f00eff8970000ceb3009c
:109d3c0000c04000c0ff9f004ff897000080fb0060
:109d4c0001d8200000804000fff8970001487800ff
:109d5c00904078007ff8970000c068000080fb00fe
:109d6c000000e9004f00de00d0bf9f005fb89700f5
:089d7c000080fa00000006005f
:020000040000fa
:109d84001200fa0080bf9f0091bf9f00a2bf9f00f6
:109d9400b3bf9f00c4bf9f00d5bf9f00e6bf9f0015
:109da400f7bf9f0010002000f0b79f000fb8970086
:109db4000000e90000004000c16d21000080400067
:109dc40010007800ee8057000d000900315878002b
:109dd400e000b1007fb097000080fa0000000600a8
:020000040000fa
:109de4000200fa0010002000f0bf9f00e40007000a
:109df400ffb8970001006000f0bf9f00a8000700b3
:109e0400ffb8970001006000f0bf9f005e010700eb
:109e1400ffb8970001006000f0bf9f0091000700a9
:109e2400ffb8970001006000f0bf9f007fb8970063
:089e34000080fa0000000600a6
:020000040000fa
:109e3c000200fa00881f7800000478000000eb0094
:109e4c00e0bf9f000800780019fa0700e0bf9f00f0
:109e5c001870a1006fb897000000e00003003200fa
:109e6c0010002000e0bf9f00020037000000eb0054
:109e7c00e0bf9f006fb897004f0478000080fa0095
:049e8c0000000600cc
:020000040000fa
:109e90000200fa008000eb00f1bf9f001070a000ec
:109ea000b0009000400190008101e800330098006c
:109eb000828f500006003600c00090008100e8004c
:109ec0003100980010002000f0bf9f000200370012
:109ed00020002000f0bf9f007fb897000080fa00ac
:049ee0000000060078
:020000040000fa
:109ee4000400fa00f0bf9f0010002000e0bf9f00b4
:109ef4007fb897000000e90000004000c15821002d
:109f040000804000900078000000eb000100e000b9
:109f14000600320000fc2f000080470035000900d5
:109f2400b05878006103b1006fb897000080fa0060
:049f34000000060023
:020000040000fa
:109f38000200fa0010002000f0bf9f0041a480003a
:109f4800e0472100ccf8070050b7800061006000ae
:109f58004300dd00018080000130a1008100700015
:109f68000180880010808000e50f500001003a0051
:109f7800ee36ef007fb897000080fa000000060078
:020000040000fa
:109f88000200fa0010002000f0bf9f00202ba8005c
:109f9800f02ba80080ff2f006e08b6005000b30019
:109fa800704388000b88a9002b88a800cca00a0061
:109fb8002a0800000080fb00ffb89700010060003d
:109fc800f0bf9f007fb897000080fa0000000600ed
:020000040000fa
:109fd8000200fa0011002000f1bf9f00bc71ef00e1
:109fe80020002000f08d880052002000028e88009a
:109ff800c231ef00218e8800c671ef00408e8800c4
:10a0080040002000508e8800cc31ef00ce31ef00a8
:0ca018007fb897000080fa0000000600ee
:020000040000fa
:10a024000614a8000634a80007f4a8001e14a8000b
:10a034001e34a8001ff4a8003614a8003634a80063
:10a0440037f4a8004e14a9004e34a9004ff4a90017
:10a054006614a9006634a90067f4a9001000200062
:04a0640000000600f2
:020000040000fa
:10a06800400420001040a1001000a1001010a10021
:10a078001070a0001060a0001050a100f1ff2c008b
:10a088001088600010f0a10000000000000000002f
:0ca0980000000000100020000000060086
:020000040000fa
:10a0a4000200fa0010002000f0bf9f00401f2000b3
:10a0b40090fd0700ffb8970001006000f0bf9f000b
:10a0c400c2e40700ffb8970001006000f0bf9f00e2
:0ca0d4007fb897000080fa000000060032
:020000040000fa
:10a0e0000a00fa00c0bf9f00d1bf9f00e2bf9f00df
:10a0f000f3bf9f0010002000b0bf9f0000c82000e9
:10a10000e880570007000900315878003fb89700f1
:08a110000080fa0000000600c7
:020000040000fa
:10a118000200fa0010002000f0bf9f002fff070088
:10a12800ffb8970001006000f0bf9f00a8fc07007f
:10a13800ffb8970001006000f0bf9f000000eb002f
:08a148000080fa00000006008f
:020000040000fa
:10a15000b0b388007836ec0000000000000000007a
:10a1600000000000000000000000000000000000ef
:10a170007216ab00020032007436ec000000fe00e4
:04a1800000000600d5
:020000040000fa
:10a184000200fa0010002000f0bf9f0040062000eb
:10a19400f3f80700f0bf9f008ce40700ffb89700b6
:10a1a40001006000f0bf9f007fb897000080fa00b4
:04a1b40000000600a1
:020000040000fa
:10a1b8000200fa0010002000f0bf9f0040132500a5
:10a1c80090b788004000200080b78800ee36ef0086
:0ca1d8007fb897000080fa00000006002d
:020000040000fa
:10a1e4000200fa0010002000f0bf9f0000002100d0
:10a1f40080f90700ffb8970001006000f0bf9f00de
:0ca204007fb897000080fa000000060000
:020000040000fa
:10a210000200fa0010002000f0bf9f0000002100a3
:10a2200058fb0700ffb8970001006000f0bf9f00d7
:0ca230007fb897000080fa0000000600d4
:020000040000fa
:10a23c000200fa0010002000f0bf9f000000210077
:10a24c0011000700ffb8970001006000f0bf9f00ed
:0ca25c007fb897000080fa0000000600a8
:020000040000fa
:10a268000200fa000000eb00f0bf9f000000210090
:10a2780011000700ffb8970001006000f0bf9f00c1
:0ca288007fb897000080fa00000006007c
:020000040000fa
:10a294000200fa0011002000f1bf9f001060a0002e
:10a2a40067f10700ffb8970001006000f0bf9f004e
:0ca2b4007fb897000080fa000000060050
:020000040000fa
:10a2c0000200fa0011002000f1bf9f001060a10001
:10a2d0005cf10700ffb8970001006000f0bf9f002d
:0ca2e0007fb897000080fa000000060024
:020000040000fa
:10a2ec000200fa0010002000f0bf9f000030200098
:10a2fc00e1fc2f00818047002900090031587800cb
:0ca30c007fb897000080fa0000000600f7
:020000040000fa
:10a318000200fa0010002000f0bf9f00a8fc070010
:10a32800ffb8970001006000f0bf9f007fb897005a
:08a338000080fa00000006009d
:020000040000fa
:10a340000000eb0051052000b1468800a10a200062
:10a35000b146880000688800bba00a00000d00001c
:08a3600061001000000006007e
:020000040000fa
:10a368000080200051052000b1468800a10a200085
:10a37800b146880000688800bba00a00000d0000f4
:04a3880000000600cb
:020000040000fa
:10a38c000200fa0010002000f0bf9f00002eef002a
:10a39c001c2eef00382eef007fb897000080fa00db
:04a3ac0000000600a7
:020000040000fa
:10a3b00041a48000e04721001ffe0700100020009c
:04a3c0000000060093
:020000040000fa
:020000040005f5
:047e0000ffffff0081
:020000040000fa
:020000040005f5
:047e2000ffffff0061
:020000040000fa
:020000040005f5
:047e30007fffff00d1
:020000040000fa
:020000040005f5
:047e38007be7ff00e5
:020000040000fa
:020000040005f5
:047e4000677fff0059
:020000040000fa
:020000040005f5
:047e4800ffffff0039
:020000040000fa
:020000040005f5
:047e5000deffff0052
:020000040000fa
:020000040005f5
:047e58000000ff0027
:020000040000fa
:020000040005f5
:047e60000000ff001f
:020000040000fa
:020000040005f5
:047e68000000ff0017
:020000040000fa
:020000040005f5
:047e70000000ff000f
:020000040000fa
:020000040005f5
:047e7800ffffff0009
:020000040000fa
:020000040005f5
:047e8000fffcff0004
:020000040000fa
:020000040005f5
:047e8800c9ffff002f
:00000001FF
